:020000040000fa
:080000001401040000000000df
:020000040000fa
:10020000140104000000000094010400000000003c
:10021000c2010400000000000e0b040000000000fa
:1002200000000400000000004f1921008079220026
:100230000001880000000000050007000c00070016
:10024000ca260200000000000040da000000fe00a4
:100250004440a90000b921000000e0000300320082
:1002600000002000a00188004440a8000000060013
:1002700020f6260001002000160037006200400032
:10028000e0804800910188009001ba0062004000bf
:10029000e0804800910188009002ba0062004000ae
:1002a000e08048000002eb006028e10005003a0011
:1002b0008301e90007003300038009000059eb00c7
:1002c000040037006128e100010032000082eb00e9
:1002d00005000700910188001001ba000200e0004b
:1002e000e6ff3a00000005009101880080027800d6
:1002f00062004000e08048003559ba008301e900ff
:10030000080032002559ba008301e90005003200d7
:100310000400e000f4ff320015d9ba008301e900bf
:10032000f1ff3a0000000600881f78000204780000
:1003300082000700080040004f047800000006001b
:100340000000fa00881f7800000478003fb9970089
:10035000ea81570080007800401920007e000700e5
:10036000800078000000e000020035000040eb0053
:1003700000f47800010078004f0478000080fa0053
:1003800000000600889fbe0080047800010078000d
:100390000204780089017800110020000f00070096
:1003a00089007800880f5000010032008000eb00c7
:1003b000010078004f04be00000006000000fa00b3
:1003c0004fb99700e881570041bf2000201c200052
:1003d000610007000080fa0000000600e487470083
:1003e000889fbe008a9fbe008c9fbe008e1f780033
:1003f00081bf9f00820078008304780000077800a6
:100400000fb997000116b8008c0578000001eb00c9
:100410000c00e00042003200010178008fb9970023
:100420000300e0003e0032000c00e0002e0032002d
:10043000c900900069009000808f500004003900ce
:1004400009007800f90007000000e00026003500f0
:1004500019a8a300060032000b017800a1002000bb
:100460000e00780036010700000578000100370013
:100470000005eb000b0478000a00e00002003200e7
:100480000e0055000004e80069009000c9019000ca
:1004900003005000880f5000020031000005eb00ff
:1004a00000047800080178008e00780003007800ce
:1004b0002200070008074700888555004900900082
:1004c00008004000c00498000a00e0000400320068
:1004d00009007800230107000000e00002003a0054
:1004e0000b00e000d2ff3a0019b8a300020032006e
:1004f000090078001b01070000c0200019006000ff
:100500000200320049009000e00498000b00560001
:100510008fb99700110009000380d800000178000e
:10052000020078004f0778004f06be004f05be005e
:100530004f04be004f00b1000000060080017800ab
:100540000200e00003003200b15978000201e90026
:10055000fdff3a00000006006200fa00889fbe001e
:100560008a9fbe000004be00020578008300780068
:100570006a80570037010700f88f9f0089979f0016
:100580000000eb00909f9f001a80fb008005fb009d
:100590000000ea00cf04de000904780050022000c9
:1005a000808f550001003a000904e9000800e000ce
:1005b0000c0034000f909700080178008a00780042
:1005c000ff8997000300010080979f008080eb0067
:1005d0000000e000900032001f98970008004000e3
:1005e000909f9f000905450050022000808f550014
:1005f000040032000b00e000e3ff3a009f989700f0
:10060000850037000000eb00f0979f00e0979f0007
:10061000d0979f00c0979f00b0979f00a0979f0022
:10062000b09f9f0009003700a0d22000008050003a
:100630000000d00001d3200001004000bf989700c7
:1006400090807000b19f9f000a05e8009a00fb00af
:10065000a0d2200001010700800078000000e00027
:10066000f1ff3a00a0c2b3009a4f10000e003a000a
:100670003fb897000080e900b0bf9f0010007800ed
:10068000a09f9f000000e00005003d000000ea0080
:10069000a09f9f003f9897000020a000b09f9f0060
:1006a0000a05e80011003700a19f9f000b003700ea
:1006b000af989700f0ff2700808f500006003200af
:1006c0006a09b9001a00fb000200400001fd2f007a
:1006d00001004000a09f9f000a05e8001a00fb00ef
:1006e000e60007000000e000f1ff3a00e0c2b300be
:1006f0009a4f1000030032000080eb00809f9f00a3
:100700001c003700a0c2b300da4f100007003a0007
:100710003fb897000080e900b0bf9f00100078004c
:10072000809f9f000a05e800120037000000eb00e0
:10073000809f9f000b0037008f989700f0ff2700e5
:10074000808f5000060032006a09b9001a00fb00d1
:100750000200400001fd2f0001004000809f9f002b
:100760000a05e8001a00fb00c40007000000e000d2
:10077000f1ff3a009a00fb0020da2000b7000700e2
:100780008040eb000000e00001003200ba40780039
:10079000817f9f0080c6b30080cf500004003a00e4
:1007a0009acf100002003a00664050000700370060
:1007b0008f789700c0c6b30080cf500005003a0084
:1007c0009acf100003003a0065404000807f9f00f0
:1007d0000a05e800a0fb2f00008447003a4178009a
:1007e00088017800ea80570060f92f000f00400070
:1007f000760107000000e00006003a00880078005b
:1008000060f92f000f004000a20007000000e00088
:100810005dff3d008080eb00010078004f05be00c9
:100820004f04be000080fa0000000600889fbe0052
:1008300000047800c0019000600090008000eb0090
:10084000808f51003b0039001801780020002900fa
:1008500000006100e20f5000090032000200780041
:100860000090a0000200e0000200350000202400fb
:1008700000007100000c78008080eb002d00370034
:100880000100260001006100810f500008003a00bd
:1008900038009000808f5100050039000800780072
:1008a000300007008080eb000000e00021003a00eb
:1008b00000c020001800600017003a00600220000d
:1008c00008004000a8049000808f540012003a00f5
:1008d00000202000260307008000780020049800f4
:1008e0000000e00005003a0029049800490498003f
:1008f0000900e80030049800060037001860a000e6
:10090000400498000020b00030049800410c98008a
:10091000510c98004d0307002800900050049800e7
:10092000380090006004980000002600180c700049
:100930008000eb00010078004f04be0000000600bc
:100940000200e0000500320090cf100004003200e9
:100950000000e8000201e900fbff3a000000eb00a4
:1009600000000600889fbe00000478000000e00040
:100970000f003a006044b8000800d00041c42000d5
:10098000608078000000e00004003200f5ff0700fe
:100990000000e00001003d008084eb000804e80056
:1009a00009007800e70f540028003c00f2ff3700f0
:1009b00010d8a30024003200a00490004000900052
:1009c000808f54000b003100090150003840900026
:1009d0000000fb0089007800050907000000e00026
:1009e000110034008084440048009000808f54003f
:1009f000f5ff390028009000400498009800780026
:100a000000c020000080600002003200a8049000b6
:100a100001003700b804900001e8a300090032008b
:100a20006904980008003700a8009000410498006d
:100a300061049800510c98001890a0000080eb0011
:100a400002003700590c98000000eb004f04be0074
:100a500000000600010878000000060090cf10009a
:100a6000050032001004e00001003a00000005001b
:100a7000d0cf1000fbff3a00000006000003b100d9
:100a8000030035009000b10001003c00100005009b
:100a9000000005000400fa00889fbe008a9fbe0087
:100aa0008c1f780000047800010678007008900020
:100ab000f8009000010050008808900001005000ec
:100ac0009808900001005000a80890000100500014
:100ad000b808900001005000c8089000810550003f
:100ae0000002220090bf9f0000032300a0bf9f00d0
:100af000081090000028a30018003a000b00e00046
:100b0000160034000b0578008a047800e20f5500c7
:100b100001003600290020000900e0000c0034002c
:100b200058009000c801900009017800ee8057003d
:100b300003000100500498008080eb000000e000fa
:100b40009c0032006808900009004000600c98008a
:100b5000090555004240a900ebff3c0078019000d8
:100b60000200e0000c00340058009000c801900022
:100b70008c00780003000100500498008080eb0096
:100b80000000e0008b00320068089000f800900040
:100b900001004000600c9800080890000000e00090
:100ba00016003400000578008a047800e20f550032
:100bb00001003600290020000900e0000c0034008c
:100bc00058009000c801900009017800ec8057009f
:100bd00003000100500498008080eb000000e0005a
:100be000740032006808900009004000600c980012
:100bf000090555004240a900ebff3c001809900090
:100c00000200e0000c003400e80090005800900062
:100c1000c801900003000100500498008080eb00a0
:100c20000000e0006300320068089000980890001f
:100c300001004000600c9800280890000000e000cf
:100c400016003400000578008a047800e20f550091
:100c500001003600290020000900e0000c003400eb
:100c600058009000c801900009017800ec805700fe
:100c700003000100500498008080eb000000e000b9
:100c80004c0032006808900009004000600c980099
:100c9000090555004240a900ebff3c0038099000cf
:100ca0000200e0000e003400e800900018089000f8
:100cb0008080400058009000c801900003000100af
:100cc000500498008080eb000000e0003900320002
:100cd00068089000b808900001004000600c98007f
:100ce000480890000000e00016003400000578007d
:100cf0008a047800e20f5500010036002900200028
:100d00000900e0000c00340058009000c801900079
:100d100009017800ec80570003000100500498009e
:100d20008080eb000000e0002200320068089000a4
:100d300009004000600c9800090555004240a900d8
:100d4000ebff3c00081090000028a30018003200c0
:100d50000b00e000160034000b0578008a047800d0
:100d6000e20f550001003600290020000900e000d4
:100d70000c00340058009000c80190000901780070
:100d8000ee80570003000100500498008080eb00c3
:100d90000000e000070032006808900009004000f1
:100da000600c9800090555004240a900ebff3c008b
:100db0008000eb00010078004f0678004f05be0070
:100dc0004f04be000080fa0000000600889fbe00ad
:100dd0008a1f78000004780001027800024578003c
:100de000830478000200fb00cf80de005002b100d7
:100df0000180b10032052000820f5000e08f5800c2
:100e000095013e00006001008d013700920137001e
:100e100091013700900137008f0137008e013700b4
:100e20008d0137008c0137008b0137008a013700b4
:100e300089013700880137008701370086013700b4
:100e400085013700840137008301370082013700b4
:100e500081013700800137007f0137007e013700b4
:100e60007d0137007c0137007b0137007a013700b4
:100e70007901370078013700ed003700760137003f
:100e80007501370074013700e9003700e8003700ca
:100e9000e7003700700137006f0137006e0137003f
:100ea0006d0137006c0137006b0137006a013700b4
:100eb00069013700680137006701370066013700b4
:100ec0004b013700640137006301370062013700ce
:100ed00061013700800037005f0137005e01370095
:100ee0005d0137005c0137005b0137005a013700b4
:100ef0005901370058013700cd003700560137003f
:100f0000150037001c003700c9003700c800370043
:100f1000c700370050013700170037004e01370077
:100f20004d0137004c0137004b013700ec00370012
:100f3000690037001f0137004701370046013700bd
:100f40002b013700440137006300370042013700ae
:100f500041013700600037006e0144001200780044
:100f6000808141009480e900010a78000009e800ce
:100f70009149780041013700a8609000c0c6b300d5
:100f800080cf50000a003a0094007800648050003e
:100f9000000a78001000be004f89de00cf91de000d
:100fa0000002be00020378008203780015003700bb
:100fb00010c7b30080cf500002003a00140178003f
:100fc0000400370014017800a0c6b30080cf5000a1
:100fd00005003a0068005100000a78003002be00a7
:100fe0002003be00070037000280e900000a7800f5
:100ff0001000780000027800cfa2de000503780020
:1010000086037800049cbe000694be00a860900091
:1010100080c6b30080cf50000f00320020c6b3005e
:1010200080cf500006003a00184078000000fb0016
:10103000cf80de0001017800820178000a003700cd
:1010400040c7b30080cf500003003200664040002c
:1010500080cf500006003a0018007800cf80de00f4
:101060000101780082017800009cbe000294be005d
:101070003800be002801be00e00f5000e08f58008d
:10108000e00f5900e08f590004003d006e0144005c
:1010900092007800d0c2b3000c0037000810900016
:1010a0000018a300040032006e0144009200780092
:1010b000b0c2b300050037000008a300570032009b
:1010c0006e0144009200780000c2b30080f4780002
:1010d0000109e80051003700a8609000c0c6b300c5
:1010e00080cf500006003a009400780064805000e1
:1010f000000a78001002be006033b8001500370007
:1011000010c7b30080cf500002003a0014017800ed
:101110000400370014017800a0c6b30080cf50004f
:1011200005003a0068005100000a78003002be0055
:101130002003be00070037000280e900000a7800a3
:101140001000780000027800050020000600200052
:1011500007002000049cbe000694be00a86090001a
:1011600080c6b30080cf50000f00320020c6b3000d
:1011700080cf500006003a00184078000080fb0045
:101180000100200002002000030020000a003700b8
:1011900040c7b30080cf50000300320066404000db
:1011a00080cf500006003a001800780001002000af
:1011b0000200200003002000009cbe000294be003c
:1011c000081090000038a300140032003800be0060
:1011d0002801be00e00f5000e08f5800e00f5900da
:1011e000e08f59000d00320080c7b300804f5500da
:1011f0000300320080c5b300804f550007003a005d
:101200006e0044009000780002c3b30082f47800be
:101210008100e8008af478000108e8007800900076
:1012200000804400600498008a4078006d00370018
:10123000a860900014017800c0c4b30080cf5000b3
:1012400005003a0068005100000a78005001be0015
:101250004000be000400370064005100000a78001e
:101260001000be00b4070700009cbe000294be0040
:10127000380090000000e00004003d006e014400d2
:1012800092007800d0c2b3000c0037000810900024
:101290000018a300040032006e01440092007800a0
:1012a000b0c2b300050037000008a30005003200fb
:1012b0006e0144009200780000c2b30080f4780010
:1012c0000109e80078009000008044006004980064
:1012d0008a40780008007800d901070067003700cd
:1012e000286090008000fb00c0062000808f500026
:1012f000230032000a003c0064005000808f500040
:101300002600320004003c0066005000808f500030
:101310000b00320021003700a00620000500370036
:1013200040072000808f50001c0032001b003c0052
:1013300063005000808f5000070032001700370014
:101340001480e900000a780010007800485c9000e2
:1013500008487800490037001480e900000a780046
:101360001002780068089000cf80de00010178004c
:1013700082017800009abe000292be003f00370052
:101380001480e900000a78001001780068089000d5
:10139000cf80de000089be00380037001480e900ed
:1013a000000a780010007800680c900008087800a7
:1013b000320037001480e900000a7800100078003d
:1013c000cf80de000101780082017800009cbe0021
:1013d0000294be00780090000080440060049800f1
:1013e00081c7b30008007800dc0007002300370045
:1013f0001480e900000a780010007800600498006a
:10140000580990000200e00002003d00850107003d
:10141000090037008000eb0049fd070080007800dc
:101420000000e000030032006800900000805000df
:101430000100370058089000100c98000f0037008a
:101440006e0144009200780050c2b30080f1780031
:101450000109e80009003700ee004400110078009f
:10146000808144000a4278008008e8000a04e00015
:1014700001003a0054c2b300844978000000eb0038
:101480004f0578004f04be0000000600889fbe0094
:1014900080047800716a8000010078000100e0009b
:1014a0000a003a0001d52000500de2001c00320075
:1014b00011007800908f5400140036008080e800fe
:1014c0001100e000faff3a00150037001100e000bb
:1014d0000600320011017800928f54000b00360094
:1014e0008280e8001100e000faff3a001001780065
:1014f00001d52000806a8000820f50000800320071
:1015000011007800908f540002003e000100780026
:10151000150037008080e800910f1100f8ff3a00b5
:10152000986a8000890f5400010031000904780096
:101530000800780099030700000178000000e0002f
:1015400005003a000000eb00890f5400060032004d
:101550000804d100f3ff3700081978000200780072
:1015600095030700cbff37004f04be0000000600c4
:10157000881f7800630440000800a1000001eb0010
:10158000800f540022003600e30f540001003e009b
:101590004800200008007800bcff070080007800a9
:1015a0000001eb000000e00019003200100178009b
:1015b0009201780064805100880f500003003100d0
:1015c00012009000800878000700370008004100f2
:1015d0008008780012029000140098001100780032
:1015e0000888510008097800910078000100e000a7
:1015f00004003200110090008180e8000000e0004b
:1016000001003a008000eb00716a88000281e80066
:10161000020078004f04780000000600881f780060
:10162000880020000800d00041c4200060807800bd
:101630000000e000010032000a0007000804e90091
:10164000f8ff3700e0b0200094033700664de20059
:1016500003003a00fbff070020c0b30066edb700af
:1016600000000600889fbe0000047800bdfc070053
:10167000800478001868a30002003200280090005f
:101680004d0307000000eb00200498003840900054
:101690000004e000050035000000fb000206070022
:1016a0000000e000010032008084eb001810900080
:1016b0000000e00008003200040607000000e0001f
:1016c000010032008084eb00181090003a030700fc
:1016d0000000eb00101498001878a3000e003200f0
:1016e0008000eb000100d00042c420000200400056
:1016f000900f1400060032008100e800e78f5000d0
:10170000f8ff3600080078002b03070010003700b0
:101710000008eb00fbff3700000ceb0000c0eb0003
:101720003044980060022000080040002004980027
:101730004004980050049800400c98006004980001
:10174000500c98007004980076004400000c98003b
:10175000090078004f04be00000006006f02b000d0
:10176000889fbe008a9fbe008c9fbe008e1f78009f
:1017700080067800d0ca2000b0b79f0080c5b300b3
:1017800080cf500002003200c2c92000b2b79f00d3
:1017900083002000c3b79f00f0c6b30080cf500085
:1017a0000a0032006940400080cf5000050032003e
:1017b000a4002000c4b79f0080c5b30080cf5000b4
:1017c00002003a0000012000c0b79f008e012000f7
:1017d0003d04be002d05be0040c6b30080cf5000c2
:1017e000030032006540400080cf50000a003a00fc
:1017f000e00f5400e08f5c00e00f5d00e08f5d00c3
:1018000005003d000800be000a01be0045060700b5
:101810000205be000004be00e00f5400e08f5c0033
:10182000e00f5d00e08f5d0003003a005d0890006e
:101830000000e0000c0032007e012000cfb09700d5
:1018400001027800cfa2de0005037800860378004d
:101850000800be000a01be00e70607003fb297007d
:1018600064407800d0e79f004fb09700cf80de0043
:101870000101780082017800d0b79f00e1b79f0096
:10188000f2b79f0083bf9f000203be000002be00ac
:101890000800be000a01be00d0060700809ebe0000
:1018a0008296be00e00f5000e08f5800e00f590014
:1018b000e08f5900220034000e00e00020003400c8
:1018c0003d00be002d01be005fb29700efb2970051
:1018d0007fb397008fbb9700cb0607000205be00c1
:1018e0000004be000e07e900e1fc2f008f804000dd
:1018f000010647005fb29700efb297007fb39700f1
:101900008fbb97000800be000a01be00cd0507008e
:101910001d0010003fb19700624e7800889ebe0007
:101920008a96be00e00f5400e08f5c00e00f5d007f
:10193000e08f5d00020034000e00e000e0ff3c009c
:10194000cfb19700e88f510010003a000d109000c1
:101950000038a3000d003200f70f570006003e00cc
:10196000e4fc2f000e024200e4c07f0000c3b3007d
:1019700080cf5000050032000e07e90000c3b3001d
:10198000e1fc2f008e80400080f07f00780117007e
:10199000920e98006d009000e3fc2f008f814100b3
:1019a0008e804100e5fa07001d0e90005d08900052
:1019b000800f560006003d000c005000800e98007d
:1019c0000d1090000040a100801698000f00370015
:1019d0000000e0000d003d000d109000740060005c
:1019e000f00f500009003a007d089000fd009000c3
:1019f000010050008d089000010050000c075000bd
:101a00004240a900010034008e0e98004f07780074
:101a10004f06be004f05be004f04be006f02b1006e
:101a200000000600800078001004e0000200320090
:101a30005104e000feff3a00008050000000060064
:101a4000ef04b000889fbe008a9fbe008c9fbe003e
:101a50008e1f7800c0af9f00a1df9f0060fa2f00ab
:101a60000f004000e0af9f00cfaa97005503be00d3
:101a70004502be0084af9f0095af9f00a6af9f00b8
:101a8000b7af9f0010c6b30080cf500016003200e1
:101a900010c4b30080cf5000130032004fab97004a
:101aa000560890000000e00003003d0060002000a8
:101ab000500b98000c0037000000e0000a003a00cc
:101ac00070c6b300afdb970080cf53000300320035
:101ad00070c4b30080cf530003003a001000200010
:101ae000cfa89700d0089800cfa89700e2fc2f005d
:101af000028047007602070080017800e20f500064
:101b000014003a00cfa99700e300900030002000b5
:101b10009009980010c6b3002fda9700804f52004a
:101b20000a00320064404000804f5200070032003b
:101b30000040e800804f52000400320002d720002d
:101b40000040e800804f520017003a0042d72000c2
:101b5000150037000000e00018003400cfaa9700fd
:101b6000e500900030002000900a980010c6b300f5
:101b70002fdb9700804f53000a0032006440400082
:101b8000804f5300070032000040e800804f5300b0
:101b90000400320082d720000040e800804f53004c
:101ba00001003a00c2d72000b25878000200780045
:101bb000b058780090487800f201370014c6b3009e
:101bc000afdb970084cf53000300320010c4b30092
:101bd00080cf530010003a004fa89700ec0040005f
:101be0001101780000c3b300005978008208e800b2
:101bf00080c7b300afd8970084cf500001003200f7
:101c000080c5b300004978004fa99700720090008a
:101c10000080e800700198000300e00003003a0033
:101c20008006eb00fda79f00d001370011c6b3006e
:101c3000afd9970081cf51000300320010c4b30028
:101c400080cf5100ad003a000ed820002fda970067
:101c5000814f5200010032001ed92000cfaa970008
:101c6000550890008006e8000000e00001003d00fb
:101c70001d0220000d06e8004fab97003604be00a1
:101c80002605be006022b8006033b8000fa8970098
:101c90009fa897002fa99700bfa997005606070095
:101ca0000000e00001003d000bf0a20088af9f00a3
:101cb00099af9f00aaaf9f00bbaf9f007fa0970086
:101cc00064005000f0a79f00efab9700805beb0033
:101cd000e7af9f003f003700c20120000300200053
:101ce00001fd2f0001804700270207000faa97007f
:101cf0009faa97002fab9700bfab9700f4af9f0050
:101d000085b79f0096b79f00a7b79f000400be004d
:101d10000601be003d0607000004be000005be002f
:101d2000670656004240a9000c0034006306070015
:101d30000002be000203be007fa897008fb097008c
:101d40001fb19700afb197005f06070080af9f00fb
:101d500091af9f00a2af9f00b3af9f00efaa970083
:101d6000e7824200e5af9f0070002000e00f5400c2
:101d7000e08f5c000d003400600020006fab970026
:101d80006f636500e6af9f00cc5bdd004455de006d
:101d90000a857300c4ddde00e00f5500e08f5d00b2
:101da000020034000000e900f4ff3b000000e900fd
:101db00005003300efa897008060eb00e1af9f00c3
:101dc0000000e900fbff3b006fa99700670141009d
:101dd000e2af9f000c00e000090034006022b80070
:101de0006033b8000fa897009fa897002fa997000d
:101df000bfa99700360607000000e000b6ff3c00d0
:101e0000efa9970064fa2f000f02420004805100ee
:101e10000006e90075fa2f0085824700e5af9f00b4
:101e20008d0f560001003d008c0678000d00e0008b
:101e30002b0035008c8f560005003d006fab9700de
:101e400066c07e00f2c0b300e74f500001003c00c6
:101e50000041eb008d00e900efab970067c0780010
:101e6000824f500006003a008d06e9008100e9002b
:101e7000efa9970063c07800824f5000faff32004c
:101e8000ef4f510004003a006faa970064c0780039
:101e90000040e80000f278000100e00007003d008b
:101ea000efaa97008502e900e5af9f008d06e800e4
:101eb0007fa0970064004000f0a79f008d00e9001c
:101ec000070033006fab970066c078000000fb008e
:101ed0006e40780000f378008100e900f9ff3b00d4
:101ee000cfab9700570890000000e0001f013d00b5
:101ef0000d00e900d00b98001c0137000fac9700d3
:101f00009fac97002fad9700bfad97006022b8003f
:101f10006033b8000800be000a01be00b605070025
:101f20000000e00005003d000bf0a20088af9f001c
:101f300099af9f00aaaf9f00bbaf9f007fa0970003
:101f4000725927000280b900026a2800130020009d
:101f50000c040700e4005000f1a79f001d003b00a7
:101f600063801000c1ff2f00010460000800ea0038
:101f7000f0a79f008004eb000800e0004700340059
:101f80000808a3000e0032006848b80042c52000cf
:101f9000020040003002be002003be000fa89700e0
:101fa0009fa897002fa99700bfa99700cd0507000c
:101fb00080af9f0091af9f00a2af9f00b3af9f0083
:101fc0000884d1008904e8000800e000ecff3c0030
:101fd000320037000100e000300034006022b80019
:101fe0000600200007ff2300b4b79f00c5b79f007d
:101ff000d6b79f00e7b79f00c0ff2f0000806000aa
:10200000f0a79f00000478008004eb001600340065
:102010000808a300100032006848b80045c5200039
:10202000050040003002be002003be003fb0970014
:10203000cfb097005fb19700efb19700a9050700f7
:102040000002be000203be00b4b79f00c5b79f00e8
:10205000d6b79f00e7b79f000884d1008904e80045
:102060000800e000eaff3c003fb29700cfb29700c3
:102070005fb39700efb397000fa897009fa8970052
:102080002fa99700bfa997000b06070080af9f00fc
:1020900091af9f00a2af9f00b3af9f004fab9700df
:1020a000d608900060c6b300afdb970080cf530026
:1020b000040032006687400060c4b30080cf530044
:1020c00003003a007fa09700008040006a074000ac
:1020d000f30f5700010034003e01200000c3b3009d
:1020e000efa8970080587800e1af9f003a003700d2
:1020f0000800be000a01be00440507000006be003d
:10210000f0b79f0081bf9f00680757004240a900b9
:102110000e003400690507000002be000203be0085
:102120000800be000a01be00670507006022b80073
:1021300046782d00771924006a05070080af9f00bc
:1021400091af9f00a2af9f00b3af9f00efa9970090
:10215000e8814100e3af9f0088002000e00f5600b7
:10216000e08f5e001100340078002000a200200003
:10217000030020007fb097008fb897007801070018
:102180006faa970005c3b30005624100e4af9f004a
:10219000f0b79f0081bf9f00e00f5000e08f580014
:1021a000020034000804e900f0ff3b000804e900e5
:1021b0000600330000c3b300efab970080637800e4
:1021c000e7af9f000804e900faff3b006fa8970003
:1021d00068004000e0af9f000e00e0000b003400fc
:1021e0000fac97009fac97002fad9700bfad970045
:1021f0006022b8006033b8000800be000a01be00cb
:10220000330507000000e000b9ff3c00efa897008d
:1022100062fa2f000f014100028050000007e90020
:1022200073fa2f0083814700e3af9f007fa09700e0
:1022300067004000f0a79f0001c3b30093cf1000d8
:102240000a003a000e07e9007fa097000000e900ad
:10225000f0a79f006faa97000402e800e4af9f0078
:1022600014427800814f5200f6ff3200cfaa970047
:10227000d508900060c6b3002fdb9700804f530055
:102280000300320060c4b300804f530004003a00e2
:102290007fa09700008040008006e8000a00370019
:1022a0008001eb0050c6b300afdb970080cf530036
:1022b0000300320050c4b30080cf530001003a0045
:1022c00013002000838640008d0f570001003d0061
:1022d0008e0678000d00e000240035008e8f560039
:1022e00006003d006fa89700e0c07e0092c3b300d7
:1022f00040c3b30080cf500001003c0002c3b300d4
:102300008d00e900efa9970063c07800824f50006c
:1023100006003a008d06e9008100e9006faa9700e7
:1023200064c07800824f5000faff320090c3b300bf
:10233000804f510004003a00efaa970065c0780072
:102340000040e80080f278000100e00007003d0056
:102350006fab97000603e900e6af9f008d06e8002b
:102360007fa097000000e800f0a79f007fa29700e1
:102370008d0178006fa99700afd897004fa89700fc
:102380000e0107004f0778004f06be004f05be0044
:102390004f04be00ef04b100000006000000e000a2
:1023a00003003400d2020700e10f400001003a00b0
:1023b0000000eb00000006000000e00036003200e4
:1023c0000081e90012027800e30f5200320036006b
:1023d0000408a30030003a00816a80000100e00098
:1023e00002003200810f5100030031000108780023
:1023f000826a88001d00370081017800110090007a
:102400000000e00008003200820f5000060031009a
:1024100080017800100090000000e000020032000f
:10242000820f5000faff39009300780001804100cc
:10243000800f510018003900820f500003003a004d
:102440008489400003017800080037009300900061
:102450000100e0000300320004004100808f5000c2
:102460000d0039001101980092019800920090002f
:102470000100e000080032009201780003004100f2
:10248000810f500004003a004e2def0010894100ea
:102490001000900010019800000006000001780074
:1024a000000020000000e000080032000000800072
:1024b0000000e000050032000000e9000000880094
:1024c0000000d0000100800002b07800000006008b
:1024d000889fbe00800478000104780031009000dd
:1024e0000000d0004501de00f07f2000800f510089
:1024f00010003a00800ceb00310090006f0060008b
:1025000008003a00210090000000e00005003a00b9
:10251000110090000000e00002003a001100e0000d
:1025200002003200200020001500370010002000bb
:10253000130037000200e00005003c0001007800b5
:10254000cf010700000178000000e0000a003c0015
:1025500038009000f10028000100600001fe230017
:10256000010070003004980020c02f00800c410052
:102570000080eb0002003700800ceb000000eb0055
:102580004f04be0000000600881f78008a9fbe002e
:10259000000478000205be00300190000200d00067
:1025a000c500de00f07f2000808f50000c003a0054
:1025b0006f00610008003a00280090000000e00071
:1025c00005003a00180090000000e00002003a0008
:1025d0001800e0001c003200200020005d003700e1
:1025e0000100e00006003a0008007800a40107009e
:1025f000800078000000eb000100e00055003c0086
:102600006108b9000a0540008b854800e07f200082
:10261000800f5500e08f5d000d0034003800900001
:102620006022b8000600200007ff2f000000e00035
:10263000030035006022b8000600200007ff2700d5
:10264000049cbe000694be0010002000410037002c
:10265000b8009000e00f5500e08f5d0005003400e9
:10266000f000280000806000c450dd000100700010
:102670003600370000002800808260006f80600014
:102680000040a0003004980061055500e0855d0021
:10269000c0fc2f00f1ff2f00800f5500818f5d00df
:1026a00006003d00350498000000eb00200498006f
:1026b00010049800000ceb00260037000a02780096
:1026c000f00f45000b003c0018009000000c780053
:1026d0002800900010049800380090002004980012
:1026e0000000eb003004980070024200f00f42003e
:1026f000f5ff34000402ea001200320018017800ed
:102700000411de00f0011200180090008300dd00cb
:10271000010c71000400de00280190008310dd0030
:1027200001007000100498000411de0038009000d1
:102730008301dd0003017100220498000400de0023
:1027400030049800380090000500700030049800b4
:102750000080eb004f05be004f047800000006002b
:102760000400fa00889fbe008a9fbe008c9fbe00b6
:1027700080bf9f0091bf9f000206be0001020700bc
:102780000001be000004be000c00be00a40407004f
:102790000fb997009fb99700000551008185590036
:1027a0000800be000a01be004f06be004f05be0075
:1027b0004f04be000080fa00000006000a00fa0084
:1027c000889fbe008a9fbe008c9fbe0000047800d8
:1027d00001457800820578008304780004067800bb
:1027e0000300e00002003c0019002000abda2000ea
:1027f00060c6b300804f55000e00320060c4b300c5
:10280000804f55000b00320070c6b300804f55005a
:102810000300320070c4b300804f550083003a00bb
:10282000e40f46008100350058089000800f5600e4
:102830007e003d000c06e80060c6b300804f5500e6
:102840001000320060c4b300804f55000d0032000c
:10285000081090000038a30004003a0058089000c7
:10286000808f540001003d00590c980058089000da
:102870000c005000500c980002003b000000eb00e0
:10288000500c98000c00e00027003c00f2014400ce
:10289000130178006800900001c3b3000170790053
:1028a0000201e80082097800580890000000e0006a
:1028b00003003c00081090000038a3000400320020
:1028c000e8009000e0c2b300807079008209e8005f
:1028d0000c00ea00d8089000808f500001003d00f5
:1028e0000106ea000c00ea00200c98000c80400071
:1028f000500c9800890f500001003d0080047800c2
:10290000680090009808900001004000390c980081
:10291000090178008b00780008f70700580890003c
:10292000090050001a003700e800900018089000d5
:102930008c8f540018003d00008040000901780091
:102940008b007800fdf60700180890000901400090
:10295000120c980009005600200c980058089000ae
:102960000000e00003003c00081090000038a300c5
:1029700006003200e8009000e0c2b30080707900e9
:10298000380890000000e800300c980058089000cb
:10299000400c9800a3003700008040000c01780034
:1029a0008b007800e5f60700180890000c00400046
:1029b000100c98008c845400580890000000e0002f
:1029c00003003c00081090000038a300060032000d
:1029d000f20144009300780068019000e0c2b30067
:1029e00000f178008109e80058089000890f500034
:1029f00001003d0080047800680090009808900075
:102a0000010040008c80450009017800cbf60700ea
:102a10001808900009004000100c98005808900019
:102a200009005000200c98007e00370070c6b300eb
:102a3000804f55000300320070c4b300804f550032
:102a400014003a0058089000808f540004003d00a4
:102a5000081090000038a30001003a00590c9800bb
:102a6000580890000000e900500c980002003b005c
:102a70000000eb00500c980051c6b30070c6b300c4
:102a8000804f55000100320051c4b3000145780069
:102a90000900370010c6b300804f550002003a000d
:102aa0000ac7b3000400370010c4b300804f5500bc
:102ab00001003a000ac5b300f20144001301780096
:102ac000680090003b7079000201e80082097800fc
:102ad000580890000000e00003003c00081090003f
:102ae0000038a30004003200e8009000e0c2b30008
:102af000807079008209e800580890000000e0002a
:102b0000100034008904e900890f500001003d00e5
:102b10008004780068009000980890000100400050
:102b2000090178008b00780084f6070018089000ef
:102b300009004000100c980058089000090050004f
:102b4000200c9800e8009000180890008085400054
:102b50008a5d78008b06e8000c00e0000400350078
:102b6000b0c2b300804d78008d05780004003700b6
:102b7000d0c2b300804d78008d0578000c06ea00c5
:102b80008004eb000c00e00009003400a1002000ec
:102b90000c0078008d0007007681540001f17f0061
:102ba000000678008904e8000000e000f7ff3c0020
:102bb000e18f540009003c0050c6b300804f55001f
:102bc0000300320050c4b300804f550003003a00a8
:102bd00000c3b300805e78008d0578000900e00036
:102be00002003a0000c3b300805d78000900e000f5
:102bf000070034008904e900f680540061c07f00ba
:102c000002c3b300825d40000900e000f9ff3c0010
:102c10006800900098089000010040000080550076
:102c2000300c98000810900074006000f00f500005
:102c30000e003a00780090009808900001004000d3
:102c4000a808900001004000b80890000100400072
:102c5000c80890008100400078089000808f5000e4
:102c600002003d0001005000000c98004f06be001d
:102c70004f05be004f04be000080fa0000000600b1
:102c8000000278003000900001002800010360007d
:102c9000150020006f0060003002980008003a0024
:102ca000240090000000e00005003a0014009000ad
:102cb0000000e00002003a001400e0003e00320094
:102cc000340090000000e0000b003a002400900067
:102cd0003002980014009000200298001400780040
:102ce00010029800000aeb00f082520034009000bd
:102cf0000000e000f5ff320034009000ef0f5000bc
:102d000014003e008001d000a40090004f08de00b7
:102d100080817100330298008100d000140190007e
:102d20004f10de0080807000210298000201d00068
:102d3000940078004f08de00000171001202980034
:102d4000010ad0008502e90003007800ef8f5100ee
:102d5000ecff3600b4019000ff8f510013003600e5
:102d60001401d10014009000cf00dd00010a7100b1
:102d70000000d100a40090004f09dd0002007000a7
:102d8000100298008100d1004f18dd008080700093
:102d9000210298000300d100300298008502e8006b
:102da00080017800ff0f5000edff3e0034009000de
:102db0006f00600030029800340090000600700040
:102dc000300298000500780000000600010178003c
:102dd00000027800110009000200d8000002fd0086
:102de0000491b900820250000400be0000000600f9
:102df0000a00fa0000027800c3202000e52020002d
:102e00000721200046212000e20f50001b003e0059
:102e1000606b8000e10f500004003200632120004d
:102e200085212000a7212000e621200013409000ea
:102e30000078a30002003a00000beb0013f0a000a2
:102e4000154090000028a30001003a0015a0a00042
:102e5000820178000200e00010003200154090006e
:102e60000008a300fdff32003100fb00800b78005a
:102e70008301e900f9ff3a00080037003000200024
:102e8000b0bf9f00c4bf9f00d1bf9f00e2bf9f00a3
:102e90006a80570000c0da006fb99700020078001e
:102ea0000080fa00000006000a00fa00110020006d
:102eb000b1bf9f00c0bf9f006a80570000c0da000a
:102ec0004fb897000080fa00000006000a00fa00e0
:102ed00051002000b1bf9f00c0bf9f006a80570013
:102ee00000c0da005fb897000080fa00000006001a
:102ef000889fbe00800478006e0de20005003a0055
:102f00000000eb00100007008080eb000000e000f4
:102f10000a003500786b8000880078000900e00026
:102f20000600320009004400070007008080eb0023
:102f30000000e00001003500880078000100780002
:102f40004f04be0000000600800078000001eb0086
:102f50000000e00003003a00c0da2000706b880037
:102f60000600370040192100808f500002003e000b
:102f7000716b8800010037000081eb0002007800cf
:102f800000000600839f68000100e00002003d0091
:102f900060001000e08018000300e00002003d0027
:102fa00060011100e08119004b0007004f00e000b4
:102fb00002003b0060001000e080180000000600e6
:102fc000889fbe008a9fbe008c9fbe000404b8008c
:102fd0000506b8008904460060854e000606b80064
:102fe0000a054600e0854e000706b8008b0546003e
:102ff000040eb800890446000a854e00050eb8008c
:103000000a0546008b854e00060eb8008b0546006b
:103010000416b8000a0546008b854e000516b80058
:103020008b054600041eb8008b0546000800be0054
:103030000a01be004f06be004f05be004f04be0091
:10304000000006000800fa00889fbe008a9fbe00ac
:10305000170007000605be000404be00e00f520082
:10306000e08f5a00e00f5b00e08f5b0008003d003e
:103070000400be000601be002a0007000205be00d3
:103080000004be000f00070026000700080007002c
:103090000802be000a03be000a000700c8ff0700be
:1030a0004f05be004f04be000080fa00000006007d
:1030b000e0b79f00f1b79f0082bf9f0093bf9f00c2
:1030c000000006006fb09700ffb097000fb997009f
:1030d0009fb99700000006006022b8000602200099
:1030e0000000d0008180d2000482d2008582d2000c
:1030f0000000a0000202520083825a0003003b003d
:103100000202420083824a000000a1000603e90097
:10311000f3ff3a0000000600efff07000400be00c6
:103120000000060060001000e08018006001190037
:10313000e081190000000600810378003e020700cc
:103140000001be006000b8000478a30013003a003c
:103150006220e10015003e000d0039008301d1001e
:103160000281d3008180d3008301d1000281d3008a
:103170008180d3008301d1000281d3008180d300fc
:103180000538b000c42add00f300b200838172006c
:1031900007f0a70003f0a00000000600f3ff2700df
:1031a000f2ff2f006110b900fbff370003ff27007b
:1031b000f7ff3700881f7800000478005001be0038
:1031c0004000be000000420081804a0002014b0026
:1031d00083814b00009cbe000294be00dc0007000f
:1031e00003003100480090000000e800400498000f
:1031f0004f04780000000600889fbe00000478009d
:103200008004eb005001be004000be00d00007006b
:103210000100310019002000040050008580580092
:103220000601590087815900009cbe000294be002f
:103230004800900009005000400498004f04be0070
:10324000000006001200fa00889fbe008a9fbe00a0
:103250008c1f78000205be000004be00f4b79f007a
:1032600085bf9f0096bf9f00a7bf9f000000eb0097
:10327000e0b79f00d0b79f00c0b79f00b0b79f00d6
:10328000a0b79f000006eb005fb197006fb09700fa
:103290008000d0000000e00015003d00e1b79f0075
:1032a000010078000200e00001003d000000a000e5
:1032b000ac00070001003d000000a000af000700c7
:1032c00001003d000000a000b200070001003d0029
:1032d0000000a0008100070001003d000000a000e8
:1032e000b20007007c805700b2ff070014003700cf
:1032f000e1b79f00010078000200e00001003d00fe
:103300000000a0009700070001003d000000a000a1
:103310009a00070001003d000000a0009d0007008a
:1033200001003d000000a0006c00070001003d000e
:103330000000a0009d0007007c805700aeff070042
:103340006fb097000000e00007003500100020007b
:10335000010020006011b80008047000898470002a
:103360000a0571008b8571000c06e800f00320004f
:10337000800f5600c4ff34006fb097000000e000db
:1033800006003d007fb297008fba97001fbb9700e1
:10339000afbb97007c80570086ff07000802be0085
:1033a0000a03be006fa897000000e00004003a0086
:1033b0002fb29700bfb297004fb39700dfb39700cb
:1033c0000400be000601be004f0678004f05be0097
:1033d0004f04be000080fa0000000600881f78003d
:1033e00018002000881f780096ff07008f87e900eb
:1033f0004f04780000000600801feb0091ff0700db
:103400008f87e900000006000800fa00889fbe00d0
:103410008a9fbe008c1f78006e00070005003d00eb
:1034200043000700300007000c003d003300070098
:103430000b003700e00f5200e08f5a00e00f5b00f6
:10344000e08f5b0006003d000400be000601be00e8
:1034500034ff07000205be000004be001c0020006f
:103460002c000700ddff07000c00e0000100320027
:103470002cff07004f0678004f05be004f04be002a
:103480000080fa00000006000800fa00889fbe00d5
:103490008a9fbe008c1f78004e00070002003d008e
:1034a0001c002000220007000f00070001003d0063
:1034b0001200070017000700cfff07000c00e00014
:1034c0000100320017ff07004f0678004f05be00cd
:1034d0004f04be000080fa000000060090b79f0075
:1034e0000100d00080b79f00e00f5400e08f5c0027
:1034f000e00f5d00e08f5d00000006000800be00e8
:103500000a01be0007ff07000205be000004be005e
:10351000000006000802be000a03be005fb097006c
:10352000efb097007fb197008fb9970000000600b9
:10353000fcfe07000100070000000600b0b79f0076
:10354000c1b79f00d2b79f00e3b79f0000000600fd
:103550000400e1000588e1000690e1000798e10021
:1035600000000600c0b79f000200d000b0b79f0067
:10357000afb097000100e00000000600b0b79f0068
:103580000100d000a0b79f009fb097000100e000ad
:1035900000000600a0b79f000100d00090b79f0078
:1035a0008fb097000100e0000000060080b79f0088
:1035b0000804d0008984d2000a85d2008b85d2000d
:1035c0005fb29700efb297007fb397008fbb970071
:1035d00000000600d9ff07000605be000404be0077
:1035e0000006eb00e00f5000e08f5800e00f59009c
:1035f000e08f5900000006008f1fd1002301070053
:103600008f87e9000000e000000006001400fa00c7
:10361000889fbe008a9fbe008c9fbe000004be0033
:103620000205be00680047000a90be000890be0078
:103630003f0107000070a7000bf0a10030432000fd
:103640009e02900080825200b0fe2f000028e10010
:1036500011003d00b0fc2f000028e10015003400ef
:103660001e0990008e0890007e0090000501b000b9
:103670000201d1008180d3000080d3008502e800e0
:10368000fbff3a000b00e00064013b00600010000b
:10369000e080180061013700f0ff2f00f1ff2700e4
:1036a0000b00e0005d013b0001002800000020004d
:1036b0005a0137006000b800580137004f89de001a
:1036c000820178005a01370007f0a2008f0137000d
:1036d000809feb00ed0007008f87e9000000e0000d
:1036e000000006002800fa00889fbe008a9fbe00e6
:1036f0008c9fbe0003866b00340107000028a300e6
:1037000064003a000128a30067003a000008a30003
:1037100062003a000108a30065003a001e00900014
:10372000be08900081064000ed3fb100f4805700d4
:10373000ee019000111ab8008e099000311bb800fc
:103740009e099000311cb800511db800f485570047
:1037500046000700fe0190003a0007008b85e80054
:103760003e0007008e09900040000700ee01900027
:10377000340007008b85e800380007008e099000b0
:10378000400007009e0990001b18b8008904400003
:103790000a854800fe019000340007008b85e80090
:1037a00038000700ee019000300007008e099000fd
:1037b0001b18b800890440000a8548000a98a30035
:1037c00008003a000402420085824a0006034b00ca
:1037d00087834b0008044c0089844c000a054d0087
:1037e0008d06e90084827200850273004c3add0088
:1037f000850272000100320015002000443ade000c
:103800001400b2004538de00cb45dd000b0070002f
:10381000c540de00cb4ddd008b8070004549de00e9
:10382000cb55dd000b017100c551de000d037800a2
:10383000b301070003f0a1000cf0a70003f0a00003
:10384000f60037001b18b8008502400006834800c8
:10385000e0834b0060044c00070037001b18b800e1
:103860000603400087834800faff37001b18b800a2
:103870008703400008844800e0844c0060054d0048
:10388000000006001b18b8000804400089844800a6
:10389000faff37000108a300dd003a005800be001f
:1038a0005801be00e3ff37000008a300d8003a002b
:1038b00009047800f9ff37002800fa00889fbe004d
:1038c0008a9fbe008c9fbe0003866b00bf0007006e
:1038d0006400e100440032006408e1004a00320064
:1038e0006100e100460032006108e1004900320059
:1038f000ec0647006000b8003d02be003d03be007c
:10390000f48657006011b8003d04be003d05be00be
:103910007d0320000b0037000000a0008d06e900a9
:10392000130032000402420085824a0006034b0065
:1039300087834b000000400081804800020149005d
:10394000838149000802520089825a000a035b0001
:103950008b835b00f0ff3b000802420089824a0033
:103960000a034b008b834b008d06e900edff3a0004
:103970008482720086827200f707b200878272002a
:1039800001003200150020001e0490003e0b900044
:1039900006035400e63fb0000368a30007003200ae
:1039a0000000a7000500a0008301d1000281d30020
:1039b0008180d3000080d3000603e8008301d1009a
:1039c0000281d3008180d3000080d3000002eb008d
:1039d0000482d2004a01070003f0a1000cf0a70006
:1039e00003f0a0008d003700640247006408e10086
:1039f000870032003400be003401be00f6ff3700fd
:103a00006108e100820032006011b8006000b80077
:103a1000f1ff370003ff270002002000fbff370003
:103a2000020ab900001bb9000200b8008100420080
:103a30008100430000000600c70ade00f107b20063
:103a4000f50fb20008003200e1cf42000200320060
:103a50000170a00024000500810f700001003200f9
:103a60000408050044000500810f700002003a00c0
:103a7000140005008502e9000000400081c04800f4
:103a8000fcff3b000170a00024000500889fbe00e1
:103a90008a9fbe008c9fbe000404be000605be00c7
:103aa000809fbe00829fbe0041010700040678008f
:103ab0000800be000a01be003d0107008406780030
:103ac0004f03be004f02be008d4f76007fb09700bf
:103ad00013003300f0ff2f008b8f6b0006003b00bc
:103ae0000d0666000c00a7000a00370007f0a600cc
:103af000100020000a003700880f5200898f5a00fa
:103b00008a0f5b008b8f5b000300390010002000e0
:103b100001003e000000200007f0a7000000ea00be
:103b20004f06be004f05be004f04be000000060059
:103b3000800078005002be005003be004439de0011
:103b4000f700b200f37f200003016100090032009a
:103b50000218e10016003a0085017200830173002b
:103b6000838173000008200015003a004000200007
:103b70001300370085017200830173008381730095
:103b800005003a0004a8be0006a8be0010002000f0
:103b90000b0037000201e9000402420085824a005e
:103ba00006034b0087834b000748a300f9ff320050
:103bb0000740a00004a8be0006a8be002000200008
:103bc00080009800920098000000060068044700fa
:103bd0000294be000094be00fc0447008694be0020
:103be0008494be0009007800d1ff07000800780027
:103bf000cfff070099007800814f70000b003b0059
:103c00000800be00fc0007004f00b10003003700b1
:103c1000f3ff2700f2ff2f006110b9004f06be002e
:103c20004f05be004f04be000080fa0000000600f1
:103c3000889fbe00830478000300e0002c0035005c
:103c400003003c0000827000040271002600320074
:103c500036432000c50020008383cf000a003900ce
:103c60000541b1008283cf00070039000541b10052
:103c70008183cf00040039000541b1008083cf006b
:103c8000010039000541b10085c353006022b8002e
:103c9000120032000a003b00848272006102600060
:103ca0008301d1000281d3008180d3000080d30042
:103cb0000603e8008743e800f7ff3a0007003700f3
:103cc00000004000818048000201490083814900d2
:103cd0000603e9008743e900f9ff3a00880007007e
:103ce00009f0a70003f0a0004f04be00000006008a
:103cf00060001000e080180060011900e0811900e8
:103d0000d3ff3b00033e2c00f7ff37002800fa00ea
:103d1000889fbe008a9fbe008c9fbe000706780069
:103d2000878669000c003b00030478008704780054
:103d300008f0a10009f0a100840f5000858f580001
:103d4000860f5900890f5c00030033000cf0a200bd
:103d500001003a000cf0a1009cff07006400e100a4
:103d60005f003200780147006408e1006100320022
:103d70006c014700748557003200be001201be007e
:103d80003a04be001a05be001e039000be0a900051
:103d90008503530006003d000004fd008104fd0082
:103da0000205fd008305fd008703ea000503780096
:103db0000df8a3000400320060041400e0841c002d
:103dc00060051d00e0851d006022b8007d03200015
:103dd0000d38e1008006eb000b0039004433dd00b4
:103de000f300b2008301730039003700848272004f
:103df0000d027800e10664008b85d1000a85d300ae
:103e00008984d3000884d3008703e900f7ff3b00cf
:103e100008004000898048000a0149008b81490060
:103e200004003b0060001000e080180060011900f1
:103e3000e08119000358a300090032008d8272004e
:103e400084827200610260008301d1000281d3008c
:103e50008180d3000080d3000603e8001b003700f8
:103e60000348a30017003a000600e00017003400e2
:103e70000603e9000d00a30000004800818048000f
:103e800002014900838149000348a3000f003a0062
:103e90000600e000090034000603e90000004000cd
:103ea00081804800020149008381490001003a00f5
:103eb0000003eb000348a300f5ff32006022b800c6
:103ec0000200370084827200618266000c000700e5
:103ed00003f0a1000cf0a70003f0a0004fff370093
:103ee000640147006408e10002003a000df8a300f5
:103ef00047ff3a003200be001201be0047ff370004
:103f00001800200057002000080453000d003d0059
:103f10000600200097fc2f000740e1001e0034003f
:103f200084827200610260008301d1000281d300ab
:103f30008180d3000080d3000804e800f8ff3a0035
:103f4000470020006104600005047400040464005c
:103f50000d00320061004000e0804800600149002f
:103f6000e081490003b8a500070032000603e8001d
:103f70006538e10004003a008301d1000281d300da
:103f80008180d3000080d300f87f20000830e1005a
:103f900003003500080378006000b8006011b80025
:103fa0004433dd00f300b20083017300000006001b
:103fb00005ff270005826100070032000428e100a8
:103fc00001003200240005000600070001003a004d
:103fd000440005000408050002000700f9ff3a004c
:103fe000140005006f82610081027000850271007b
:103ff0008502720000000600e48240001078a300f1
:1040000007003200640240001178a3003400be00b3
:104010001401be00040032000330a70000000600b7
:104020003500be001501be000330a00000000600f0
:104030000200fa00881f78004079280051a820006b
:10404000604588007145880030f92e00414121000b
:10405000804588009145880020002000000f7800ee
:10406000d00120009e0f100018003c009e00780038
:10407000400020000008b800c28a2000020440006e
:104080001e0078006103b900431c2e0063009000fd
:104090000032b8007300900000b0b900050178004c
:1040a00000014100630090000780b9000001410059
:1040b000820278004079280051a82000001c4200ac
:1040c00001944a001e0fe800e5ff370010002000b1
:1040d000504988000000eb00604988002000200063
:1040e000704988000000eb00000f7800d00120002c
:1040f0009e0f100008003c001e0078000000d00059
:1041000002932000820040000000eb00800878004d
:104110001e0fe800f5ff37000000eb00604b880041
:104120000000eb00704b88000000eb00904b880013
:104130000000eb00804b880020002000a04b88008e
:10414000007d2000b04b880040062000c04b880056
:104150000000eb00d04b8800b0042000e04b88004a
:1041600020022000f04b8800e0012000004c880075
:10417000d0012000104c8800e0272800010020001a
:104180002049880031498800d04e210040498800ec
:1041900020002000204c880010002000304c8800b7
:1041a00010002000404c88000000eb00504c8800bc
:1041b00030002000604c880000502900a1ab200096
:1041c000804c8800914c8800509d21000100200007
:1041d000a04c8800b14c880040082000010020005d
:1041e000c04c8800d14c88000078200001002000dd
:1041f000e04c8800f14c8800700120000100200094
:10420000004d8800114d8800700120000100200041
:10421000204d8800314d880020032000404d88004b
:1042200030c0b300aae9b70030c0b300abe9b700b3
:1042300010c0b300ace9b70010c0b300ade9b700df
:1042400010c0b300aee9b70010c0b300afe9b700cb
:1042500010c0b300b0e9b70010c0b300b1e9b700b7
:1042600010c0b300b2e9b70010c0b300b3e9b700a3
:1042700010c0b300b4e9b70010c0b300b5e9b7008f
:1042800013002000a28a2000e11f2f00f007200069
:104290009d100700504580000000e8005045880050
:1042a00012002000e11f2f00f0072000a3100700dc
:1042b00013002000e21f2f00f1072000a08a200039
:1042c000bf1007004f0478000080fa0000000600cd
:1042d0000400fa000000eb00704c88000000eb00c6
:1042e000000f7800100720009e0f100024003e00f1
:1042f000000720009e0f100008003e001e007800fe
:104300000000d000c28a200082004000704c800073
:1043100011004000704c880003003700704c800092
:104320000000ea00704c88001e0078000000d000f9
:1043300002002f008200400012002000f007200041
:104340007e100700100798001e0078000000d000c3
:1043500001002f00010140001e0078000000d00085
:10436000c18a20000100400013002000f107200056
:1043700093100700100798001e0fe800d9ff3700c0
:104380008e09f8001e019000821f78001e00780040
:10439000801f780080282e00801f780007f007001b
:1043a000e88757000080fa00000006000600fa00c7
:1043b0000000eb00200798000000eb00000f7800e1
:1043c000100720009e0f100015003e001e00780010
:1043d0000000d000c18a2000010140001e007800ca
:1043e0000000d00003002f008300400013002000d5
:1043f000f007200044100700100798001e00780006
:104400000000d000c28a2000820040002e009000f0
:1044100011004000200798001e0fe800e8ff370059
:1044200013002000a28a2000e11f2f00f0072000c7
:10443000351007002e0090000080fa0000000600f2
:104440000400fa000000eb00d04d88000000eb00f3
:10445000000f7800500120009e0f100024003e0045
:10446000410120009e8f100008003e001e007800d1
:104470000000d0000299200082004000d04d800052
:1044800011004000d04d880003003700d04d80005f
:104490000000ea00d04d88001e0078000000d00027
:1044a00002102f008200400012002000f0072000c0
:1044b00022100700100798001e0078000000d000ae
:1044c00001102f00010140001e0078000000d00004
:1044d000019920000100400013002000f107200096
:1044e00037100700100798001e0fe800d9ff3700ab
:1044f000ba09f8001e019000821f78001e007800a3
:10450000801f7800102b2e00801f7800abef070073
:10451000e88757000080fa00000006000600fa0055
:104520000000eb00200798000000eb00000f78006f
:10453000500120009e0f100015003e001e00780064
:104540000000d00001992000010140001e00780009
:104550000000d00003102f00830040001300200053
:10456000f0072000e80f0700100798001e007800f1
:104570000000d00002992000820040002e00900030
:1045800011004000200798001e0fe800e8ff3700e8
:104590002e0090000080fa00000006000e00fa00d5
:1045a000000f7800110798009e0090004006200040
:1045b000008ab9001e0078006101b9000400be0045
:1045c00070fa070030079800410798004206200063
:1045d000030020003e009000ce009000000051003b
:1045e0008180590050079800610798005e00900094
:1045f000ee009000e00f5000e08f580004003c00f7
:10460000100020000100200050079800610798006a
:10461000100320009e0f1000150034003e00900093
:10462000ce009000420620000202b8000001eb001c
:104630000283b9000501780006014100430620000d
:104640000388b90000014100820278000071220055
:104650000100200004004000858048005e019000b9
:10466000ee01900047fa070020079800020037008b
:104670000000eb00200798002e0090000080fa0058
:10468000000006000400fa00b00020006f0e0700d2
:10469000cf80de00e24c80000202b800f24c8000c5
:1046a0000283b9000501780006014100e34c800057
:1046b0000198b9000001410082027800048fbe0019
:1046c0001e00be004008de0001002000b04388004c
:1046d000b0438000b20a07000080fa000000060024
:1046e0000200fa00c1438000207520000088b90054
:1046f0004008de0001002000f0448800f044800003
:10470000a70a07000080fa00000006000000fa0077
:104710003408e20002003a00f1ff07000100370010
:10472000d8ff07000080fa00000006000200fa002f
:104730003408e20026003a00b02d2e00a50b070039
:1047400031448000204d8000000ab80031448000d0
:10475000304d80000088b90005017800000141005b
:10476000214d8000404480000088b90000014100d4
:104770008202780040a8de00cf80de00000f7800c3
:10478000504480009e0f1000040034001e0078008a
:104790005044880060042000604488006044800029
:1047a0000000e900604488008c08e20004003a0040
:1047b00060042000604488001e0078005044880097
:1047c0007107200050448000bb0c07000600370032
:1047d000f02d2e007f0b07000000eb0050448800f6
:1047e00060042000604488000080fa000000060099
:1047f0000000fa003408e20018003a00900020009f
:10480000120e0700cf80de00a24c80000202b8002a
:10481000b24c80000283b900050178000601410016
:10482000a34c80000198b900000141008202780089
:1048300040a8de00cf80de00e0438800802e2e00fe
:10484000640b070021002000e04380009a0c070061
:10485000b02e2e005f0b070002003700d02e2e0076
:104860005c0b07000080fa00000006000200fa005e
:104870000000eb00000f7800a00020009e0f100049
:104880000c003c00821f2e009e007800400020009b
:104890000008b80000014100d0408000e1408000e5
:1048a000b20f5000a28f5800020035001e0fe80022
:1048b000f1ff37001e007800604188000080fa0098
:1048c000000006000000fa00e8ff070060418000d9
:1048d000a19a2000010040001080fb004e00dd0086
:1048e0005041880041222e00604180000000d0002d
:1048f0000100400010007800e04d8800e14d80008c
:104900005041800000807000e04d8800d24080005f
:10491000e3408000b0602b0001b62000800f510002
:10492000818f590004003400e04d80000108200010
:1049300001007000e04d88008809e20004003200a8
:10494000e04d80000104200001007000e04d88006f
:104950007009e20004003200e04d800001022000f6
:1049600001007000e04d88007209e200060032008c
:10497000404c8000e10f500003003a00e04d800001
:104980000040a000e04d88006e09e2000300320004
:10499000e04d80000030a000e04d88007409e20086
:1049a00003003a00e04d80000020a000e04d8800a8
:1049b000104180000000d000019320000100400061
:1049c00011002000908f100003003200e04d8000a5
:1049d0000010a000e04d8800104180000000d000d1
:1049e000019320000100400011002000908f100072
:1049f00003003c00e04d80000000a000e04d880076
:104a0000e04d8000cf1107000080fa000000060092
:104a10000200fa0000000000cfc2bf000080fb00cf
:104a20004600de000080fb0061006000e10f5000e6
:104a30005c003a00d0002000840d0700c0438800cd
:104a4000c0002000810d0700d0438800c1438000d2
:104a5000c04380000088b900f0438800014488000a
:104a6000d1438000d04380000088b9001044880002
:104a700021448800f24380000344800010448000f9
:104a8000214480000000510081805900304488009a
:104a9000414488000040eb000e0907001bff07009f
:104aa000b02d2e00cb0a070031448000204d80003d
:104ab000000ab80031448000304d80000088b90001
:104ac0000501780000014100214d80004044800034
:104ad0000088b900000141008202780040a8de0091
:104ae000cf80de00000f7800710720001e007800e4
:104af000f10b070000c4b300f6080700602f2e007a
:104b0000b40a070060418000a19a20000100400023
:104b10001004e00003003a0000022000860a0700ab
:104b200002003700d0022000830a070060418000a5
:104b3000a19a20000100400010407800330c0700cb
:104b400020302e00a30a070060418000a19a2000b7
:104b5000010040001080fb00000f7800a000200042
:104b6000120e07001e0f1000300020009e0f1000d4
:104b70000200340030002000000f78001e00e0002a
:104b800002003d000000eb00000f78006041800053
:104b9000a19a2000010040001e48780049ff07004c
:104ba0009dff370026fe0700f60d07000080fa0083
:104bb000000006000000fa003208e20002003200a5
:104bc00093ff070040003700604380000000a20010
:104bd000604388006c08e20004003a00414d800008
:104be000c0f621002510070003003700414d80006a
:104bf000108f210021100700c0080700004b200083
:104c0000b0678800cfc2bf000080fb004600de0016
:104c10000080fb0061006000e10f50002a003a00b4
:104c20000040eb00ab080700b0678000c212200014
:104c3000110009000280d800801f780060302e002b
:104c4000801f7800c0832000bded0700e487570077
:104c5000c08320005f0a070000c4b3009d0807005e
:104c60006c08e2000300320090312e00590a070060
:104c700002003700a0322e00560a0700f60ce200b0
:104c8000e0ff3a00404d80008000d000e055220057
:104c9000fa0f0700404d80000000d000190d0700fa
:104ca0008bfd0700550f0700b0332e00801f7800e2
:104cb000c2ed07008f87e90020002000110d0700da
:104cc000cfa2a900ffff37000080fa000000060015
:104cd0000200fa008908070080362e003d0a07000e
:104ce00000c4b3007b08070090372e00390a070084
:104cf0001d0c07000000e000110032002a0c070024
:104d0000004f7800a1002000904f2100db0f07002a
:104d10001e407800050c070000c4b3006d080700b2
:104d2000a0382e002b0a07001e80fb00020a070095
:104d300040392e00270a07001e407800040a0700a9
:104d4000cfc2bf000080fb004600de000080fb00f9
:104d500061006000e10f5000e5ff3a000080fa00ba
:104d6000000006000000fa00c04b80003d0f070065
:104d7000d04b8000304588000080fa00000006001b
:104d80000000fa000000eb00360f07000080fa0078
:104d9000000006002600fa00889fbe008a1f7800e7
:104da000f0f32f00001688000000eb0010168800ba
:104db00030e72f00301688000000eb004016880016
:104dc000e0012400601688000000eb0070168800e7
:104dd0000000eb00901688000000eb00a016880091
:104de00080e12f00f01688000000eb00001788001b
:104df00000082100201788000000eb003017880011
:104e0000cfa2a80040442500a0048800d00e0700cf
:104e1000b30d07006000b800990d07004079280025
:104e200051a82000960d070050552500515525002a
:104e300020408800314088002003200080678800df
:104e4000c0d42100404088000000eb0050418800a1
:104e50000000eb00e04d8800ac100700e04d800042
:104e6000b81007002d080700760807002308070080
:104e700090392e00d7090700a0192e00d509070088
:104e800000c4b30013080700403a2e00d109070000
:104e9000890b0700cc190700503b2e00801f7800bb
:104ea00046ed07008f87e900a0192e00801f7800cb
:104eb00042ed07008f87e900d03c2e00801f78006c
:104ec0003eed07008f87e900101a2e00801f780042
:104ed0003aed07008f87e900603d2e00801f7800c3
:104ee00036ed07008f87e9000808f800e03f2e0044
:104ef000801f780031ed0700e487570060412e00e5
:104f0000dd190700420c070060432e00b1090700bd
:104f10000000eb005043880080bb2000b067880091
:104f2000cfc2bf000080fb004600de000080fb0017
:104f300061006000e10f500020003a00f60ce20032
:104f4000f7ff3a009f0e0700c1122000e055220033
:104f50004a0f070000c4b300de070700f0432e002d
:104f60009c090700100020005043880020c7210042
:104f7000711c27002040880031408800cfc2bf004c
:104f80000080fb004600de000080fb006100600046
:104f9000e10f5000f9ff32000040eb00cd070700a1
:104fa00000452e008b09070000c4b300c9070700a5
:104fb00010462e0087090700d9ff370057fd07006c
:104fc00030079800f9fc070040079800aa08f8008d
:104fd0004e009000801f7800be009000811f780076
:104fe00020472e00801f7800f4ec0700e887570068
:104ff0003e0090000000e00003003a004e009000e8
:105000000000e0000800320018120700904b2e004c
:10501000801f7800e9ec07008f87e90004fc070097
:1050200007fd0700aafc0700b04b8000930e0700a5
:10503000c04b80008b0e0700cb0c07000000eb007c
:10504000604388000000eb00204388000000eb0074
:10505000304388000000eb00304388000000eb0084
:10506000904188000000eb00804188006249800088
:105070001241880010418000e10f5000020034000e
:105080000000eb001041880011418000400020002a
:105090000008b800c38a2000030040001001be00d1
:1050a000d2408800e3408800d0408000e14080008a
:1050b000f30c070008140700007d2000110c070006
:1050c0008e070700931707003e0e070040012000df
:1050d0000c0c0700404d80008000d000904f210054
:1050e000e60e07006a08e2000100320038100700ef
:1050f00000000000cec2bf000080fb004200de00c6
:105100000080fb00610060000000e00012003a0037
:105110000040eb006f070700a04e2e002d0907008e
:1051200000c4b3006b070700b04f2e002909070029
:10513000c3c2bf000080fb004400de000080fb0013
:10514000610060000000e000eaff3a00b8fb0700e1
:10515000bbfc07005efc0700614c80008000200063
:105160000008b800c3232e0000804100801f780093
:105170008c09f800c0502e00801f78008fec0700cb
:10518000e6875700604c8000d90a0700604c800019
:10519000e30f50000b003200614c800080002000c3
:1051a0000008b800c4232e0000004200801f7800d1
:1051b0008c09f80070532e00801f78007fec0700e8
:1051c000e6875700c3c2bf000080fb004500de0039
:1051d0000080fb00610060000000e00001003a0078
:1051e000bbfe0700e90a070038190700ddfe0700cb
:1051f000c8c2bf000080fb004600de000080fb004c
:10520000610060000000e000030032001000200098
:10521000a0418800030037000000eb00a041880097
:10522000d0fe07006049800010418800704980006e
:10523000e20f500027003a00a0418000e10f50002b
:1052400006003a0010418000e10f500008003400d1
:105250000000eb001041880005003700104180007d
:10526000e10f5000020034001000200010418800bf
:1052700060498000e20f500009003a009049800028
:10528000e20f500003003a00100020008041880027
:105290001c0037000000eb00804188001900370037
:1052a000104180000000d000019320000100400068
:1052b00022002000900f110003003a00100020008f
:1052c000804188000f0037000000eb00804188001b
:1052d0000c003700104180000000d0000393200034
:1052e0000300400024002000900f120003003a0049
:1052f0001000200080418800020037000000eb0011
:1053000080418800104180000000d00001932000ff
:105310000100400032002000900f11000f003a0001
:105320003408e20009003a00ca62a8003208e2002c
:105330000f003a001000200090418800414d80008d
:10534000904f21004d0e070009003700ca62a900e6
:105350000000eb0090418800050037003208e200b1
:10536000030032000000eb0090418800ca62a900ef
:105370003e4de200660032006408e20064003a003c
:105380000040eb003eedb7006c08e2005f003a0021
:1053900074fe07000a08e2001d003a001141800077
:1053a000400020000008b800c38a200083044000a9
:1053b00011418000400020000008b800c48a20008d
:1053c00004044000ef0b07006103b900421c2e00eb
:1053d00051498000400020000008b80080014100d1
:1053e0001332b8001300900000b0b9000501780036
:1053f00000014100130078000780b900000141005e
:1054000082027800b81c4200a8944a001c003700b1
:1054100011418000400020000008b800c28a20002e
:105420008204400011418000400020000008b800c4
:10543000c38a200003044000d20b07006103b900b7
:10544000c21a2e0061408000400020000008b80011
:10545000800141001332b8001300900000b0b90081
:105460000501780000014100130078000780b900b1
:105470000001410082027800b81c4200a8944a0052
:1054800011418000400020000008b800c48a2000bc
:10549000040140002040800031408000b20f100025
:1054a000a28f180008003400114180004000200045
:1054b0000008b800c28a200002004000224080009c
:1054c000334080000288be0011418000400020006f
:1054d0000008b800c38a2000030040001000be008e
:1054e000e00f5000e08f580009003d00114180009e
:1054f000400020000008b800c48a200004014000d9
:105500006000b8000089be00010037009d0b070055
:1055100011418000400020000008b800c28a20002d
:10552000020040001001be00d2408800e340880025
:1055300011418000400020000008b800c38a20000c
:10554000030040001001be00f240880003418800c3
:105550006c09e20027003200f0002000bb0a0700bf
:1055600020079800ae00900010832000808f50002c
:10557000050034002e009000e37c2f000300400063
:10558000200798000b003700ae009000e07c200060
:10559000808f500005003c002e00900024832f00d7
:1055a0000400400020079800020037000000eb00d4
:1055b00020079800ae009000800120000088b9000c
:1055c0002041880031418800a0418000e10f500057
:1055d00008003a002041800031418000d240800024
:1055e000e34080000201400083814800d2408800ef
:1055f000e3408800104180000000d00003932000a9
:105600000300400024002000900f120012003a0016
:105610003408e20010003a00d2408000e3408000ed
:1056200020498000314980000000510081805900ec
:10563000d0408800e1408800f240800003418000b3
:1056400020498000314980000000510081805900cc
:10565000f040880001418800d0408000e140800097
:10566000870b070097fc07003408e2000d003a00a2
:10567000104180000000d000019320000100400094
:1056800012002000900f110003003c00104c80001d
:10569000e60c07000900370020032000e30c070098
:1056a00006003700a04b80000000d000c397200008
:1056b0000300400010007800dc0c07003408e20012
:1056c00031003a00d0002000600a0700c043880083
:1056d000c00020005d0a0700d0438800c14380005d
:1056e000c04380000088b900f0438800014488006e
:1056f000d1438000d04380000088b9001044880066
:1057000021448800f243800003448000104480005c
:1057100021448000000051008180590030448800fd
:1057200041448800d1438000c04380009bfb0700b8
:10573000c04488009c08e20003003200e04480007e
:105740000000e900e0448800c1448000c01220004d
:10575000808f5000090034009c08e20007003a00e6
:105760000000eb0020438800200020003043880028
:1057700010002000d0448800050037000000eb0036
:10578000d044880002003700800c2000e0448800ec
:10579000e00020002d0a07000045880001002100dc
:1057a0000045800000805000200798002e009000e7
:1057b0004015b00020079800ae0090002e00900029
:1057c0000088b900300f9800410f98003e08900003
:1057d000ce0890004108de0001002000200798005c
:1057e0002e00900074004000200798002e029000c8
:1057f00084678800204c8000c04188008a09e2004c
:10580000160032003408e20014003200b043800079
:105810008080e800004580004680de00808f5000d8
:10582000080034006e08e20006003a00770c07001a
:10583000401f2000104588000000eb002045880034
:105840000d003700a208e2000b003a006b0c0700c5
:105850001000200020458800070037000000eb0002
:10586000204588006e08e20002003a00670c07003d
:1058700001003700610c0700c3c2bf000080fb00bd
:105880004500de000080fb00610060000000e000d9
:105890005a003a0033fd0700803e2000b0678800c0
:1058a0006408e20007003a0030438000e40f500033
:1058b00004003a00414d8000c0f62100ef0c0700c3
:1058c0000d00370020438000e10f500007003a0030
:1058d00040438000ed0f500004003a00414d80002d
:1058e000c0f62100e50c070003003700414d8000a1
:1058f000108f2100e10c070040062000010a07007c
:10590000c3c2bf000080fb004500de000080fb003a
:10591000610060000000e00008003a00f60ce200c0
:10592000f7ff3a00414d8000a00020000088b90038
:1059300080007800c0f62100d00c0700f60ce200d1
:1059400013003a00204380000000e8002043880054
:1059500020438000e10f5000020034000000eb0003
:105960002043880000000000c3c2bf000080fb008d
:105970004500de000080fb00610060000000e000e8
:10598000f9ff320040062000de090700130037004f
:105990006408e20009003a00304380000000e8009b
:1059a0003043880030438000e40f50000b00340087
:1059b0000000eb00304388000800370040438000bf
:1059c0000000e8004043880040438000ed0f500095
:1059d000020034000000eb0040438800690a070021
:1059e000c3c2bf000080fb004500de000080fb005a
:1059f000610060000000e000f9ff3200c3c2bf0098
:105a00000080fb004400de000080fb0061006000bd
:105a10000000e0003c003a00d2fc07005049800042
:105a2000e20f500004003a00414d8000c0f6210012
:105a3000920c070003003700414d8000108f2100b9
:105a40008e0c0700803e2000b067880040062000d2
:105a5000ac090700c3c2bf000080fb004400de00a9
:105a60000080fb00610060000000e00008003a00d8
:105a7000f60ce200f7ff3a00414d8000a000200044
:105a80000088b90080007800904f21007b0c07004f
:105a9000f60ce2000c003a0040002000504988005b
:105aa000c3c2bf000080fb004400de000080fb009a
:105ab000610060000000e000f9ff320040062000b5
:105ac000900907000800370050498000e20f50009d
:105ad00003003a00100020005049880002003700ff
:105ae000200020005049880000000000c3c2bf0011
:105af0000080fb004400de000080fb0061006000cd
:105b00000000e000f9ff3200cec2bf000080fb00c1
:105b10004400de000080fb00610060000000e00047
:105b200017003a008ffc07006c09e2000600320003
:105b3000414d8000c0f62100500c07000000eb0032
:105b4000604b880005003700414d8000108f210018
:105b50004a0c070010002000604b8800400620001f
:105b600068090700cec2bf000080fb004400de00d1
:105b70000080fb00610060000000e000f9ff3200df
:105b8000cec2bf000080fb004300de000080fb00af
:105b9000610060000000e000b6003a003408e20056
:105ba000b40032006ffc070070498000e20f500023
:105bb0004b003a0060498000e20f500004003a00b8
:105bc000414d8000c0f621002c0c07000300370077
:105bd000414d8000108f2100280c07000000eb00d1
:105be000a0498800803e2000b06788004006200061
:105bf00044090700cec2bf000080fb004300de0066
:105c00000080fb00610060000000e00008003a0036
:105c1000f60ce200f7ff3a00414d8000a0002000a2
:105c20000088b90080007800c0f62100130c07003e
:105c3000f60ce20021003a002208e2000b003a00d4
:105c40006245800073458000824588009345880046
:105c5000834980009349880000c4b3009d04070075
:105c600010562e005b0607000a00370080458000b2
:105c70009145800060458800714588009149800009
:105c80008149880000c4b3009204070020572e0009
:105c900050060700400620001a090700cec2bf00c8
:105ca0000080fb004300de000080fb00610060001c
:105cb0000000e000f9ff32001e003700604980005c
:105cc0000000e8006049880060498000e20f500051
:105cd000180034000000eb00604988001500370010
:105ce000704980008000e90060498000810f500009
:105cf00004003a00414d8000c0f62100df0b070090
:105d000003003700414d8000108f2100db0b07009e
:105d1000604980000000e800604988006149800017
:105d200070498000808f5000020035000000eb00b9
:105d30006049880093090700000f7800cec2bf00b9
:105d40000080fb004300de000080fb00610060007b
:105d50000000e00045003a00200120009309070000
:105d6000200798002e0090000000e000f3ff3200b2
:105d7000614980002e00900000804000604988004a
:105d80006149800070498000808f50000300350019
:105d9000704980000000e900604988002c09e20099
:105da00002003d000000eb006049880000c4b30021
:105db000480407002a81200061498000400020003b
:105dc0000008b800c28a2000020340001600be008e
:105dd0004f8ade00cfa2de001600be00040178006c
:105de00084017800844c8000954c80004facde002c
:105df000cfc4de00844c8000954c800008037800fe
:105e0000880378008ff40700009dbe000295be0055
:105e1000208120005001be004000be00140220007e
:105e20008381d1000281d3008180d3000080d30020
:105e30000402e900faff3a00300f9800410f980081
:105e40003e089000ce089000d706070030582e007c
:105e5000e0050700604980001004b000b6050700a7
:105e600080582e00db050700b4ff37004509070006
:105e7000000f7800cec2bf000080fb004200de00b1
:105e80000080fb00610060000000e0002c003a0090
:105e90003408e2002a003200b2fb07001041800003
:105ea0000000d000019320000100400032002000db
:105eb000900f110004003a00414d8000c0f621000f
:105ec0006e0b070003003700414d8000108f21004a
:105ed0006a0b0700104180000000d00003932000ef
:105ee000030040001008e800104180000000d000ce
:105ef000049320000400400031002000908f100027
:105f000006003400104180000000d0000293200001
:105f1000820040000000eb0080087800400620006e
:105f200078080700cec2bf000080fb004200de0000
:105f30000080fb00610060000000e000f9ff32001b
:105f4000cec2bf000080fb000000d1000080fb003b
:105f5000610060000000e00021003a0081fb0700c2
:105f60007409e20004003a00414d8000c0f62100af
:105f7000420b07000a003700a04b8000e20f5000e0
:105f800004003a00414d8000108f21003b0b0700b8
:105f900003003700414d8000904f2100370b070070
:105fa000a04b80000000e900a04b88007409e200cb
:105fb00002003d0020002000a04b88004006200089
:105fc00050080700cec2bf000080fb000000d100d7
:105fd0000080fb00610060000000e000f9ff32007b
:105fe000a808e200030032000000eb0040458800f2
:105ff00063fb07000040eb00b6030700234380006b
:10600000131798001e129000e10f52002201320077
:106010001e109000e10f5000030034009e1090000d
:10602000e28f500034033200b8f907003243800099
:10603000620f9800ee099000e28f51004f0032008d
:106040006e0a9000e20f520007003c006e089000bc
:106050000000e0000a003200ee089000e18f5000de
:1060600044003200060037006e099000e30f510033
:1060700052003200ee099000e48f51008600320099
:10608000104180000000d000049320000400400074
:106090001000e00004003a0070c0b300bf03070026
:1060a000b0582e004b050700104180000000d000c2
:1060b000019320000100400012002000900f110009
:1060c00004003a0070c0b300b4030700f0582e007b
:1060d00040050700104180000000d000039320001d
:1060e0000300400024002000900f120004003a003a
:1060f00070c0b300a903070030592e003505070012
:10610000104180000000d0000193200001004000f9
:1061100032002000900f110002003a0070592e004a
:106120002c0507003408e20003003a00c0592e0095
:1061300028050700590037007409e20002003a0000
:10614000105a2e0023050700a04b8000e10f5000dd
:1061500002003a00605a2e001e050700a04b800086
:10616000e20f50004d003a00b05a2e00190507000a
:106170004a0037006df90700480037003408e20094
:106180000b003a00005b2e00120507009808e200a1
:1061900003003a00405b2e000e0507003f00370069
:1061a00021002000c0448000430607003b00370068
:1061b000a05b2e000705070038003700a000200074
:1061c000a2070700cf80de0092438000a343800037
:1061d000020140008381480092438800a343880065
:1061e000006b80000000e800006b8800006b8000fe
:1061f000ef0f5000290034000000eb00006b880016
:1062000090438000a1438000cc09dd004400de0003
:1062100000807100c488de00c24c80000202b80019
:10622000d24c80000283b9000501780006014100cc
:10623000c34c80000198b90000014100820278003f
:10624000340f9800450f98006000b8009043880014
:10625000a14388003e089000ce089000480add0067
:106260004800de0000007200c808de00804388009d
:1062700070c0b30049030700305c2e00d50407004e
:1062800021002000804380000b060700505c2e0098
:10629000d00407000100370055f9070000c4b3001f
:1062a0000c0307000e08e20024003a002a812000b7
:1062b000f0408000014180004f8ade00cfa2de0066
:1062c000f0408000014180000401780084017800e2
:1062d000844c8000954c80004facde00cfc4de00c3
:1062e000844c8000954c8000080378008803780077
:1062f00054f30700009dbe000295be0020812000df
:106300005001be004000be00140220008381d10075
:106310000281d3008180d3000080d3000402e90011
:10632000faff3a00300f9800410f98003e089000a5
:10633000ce0890009c0507000a003700f04080005e
:1063400001418000809fbe00705c2e00801f78009d
:10635000c0832000fae70700e6875700c0832000cb
:106360009c0407006c08e20048003a00604b800083
:10637000e10f500027003a00a0418000e10f5000db
:1063800024003a002a812000204180003141800011
:106390004f8ade00cfa2de00204180003141800024
:1063a0000401780084017800844c8000954c8000c2
:1063b0004facde00cfc4de00844c8000954c8000e2
:1063c00008037800880378001ef30700009dbe00d4
:1063d0000295be00208120005001be004000be009a
:1063e000140220008381d1000281d3008180d30078
:1063f0000080d3000402e900faff3a002007980069
:10640000c05c2e00730407002e0090006d0507008d
:106410005902370060498000e20f500006003a0040
:1064200070498000e20f500003003a00f05c2e003b
:10643000680407000500370030582e006504070087
:10644000604980001004b0003b0407005049800000
:10645000e10f500002003a00505d2e005d0407007d
:1064600050498000e20f500002003a00805d2e008b
:106470005804070050498000e40f50003e023a00e3
:10648000b05d2e00530407003b023700e05d2e0094
:10649000500407003802370032fa07000040eb00d2
:1064a0008c02070099f8070070c0b300bb02070018
:1064b000605e2e004704070000c4b3008502070099
:1064c000404380006101b900720f980003179800e3
:1064d000d0002000010020007e0990008e11900065
:1064e000800f5100818f590011003e007e089000fe
:1064f0008e109000006001000d0037001e00370074
:10650000720037008300370094003700a500370081
:10651000c80037001f013700300137004b0137003a
:106520006601370085013700a8013700ca0137002e
:1065300094070700000f78001e00e00002003400fe
:1065400010002000704b88001e00e00002003d009b
:106550000000eb00704b88006e09e200030032007f
:10656000e05e2e001b04070003023700f05f2e00e0
:106570001804070000023700a04b80000000d00084
:10658000c197200081044000a04b80000000d00093
:10659000c297200002044000a000200083070700eb
:1065a000980c1000a04b80000000d000c397200082
:1065b00003014000c1272e00a04b80000000d00046
:1065c0000100400012017800900f510009003d00c9
:1065d000a04b80000000d000c497200004014000c0
:1065e000c1272e00a04b80000000d0000100400019
:1065f00010097800a04b80000000d000c197200057
:106600000101400021282e00a04b80000000d00096
:106610000100400012017800900f51000900340081
:10662000a04b80000000d000c39720000301400071
:1066300021282e00a04b80000000d0000100400067
:10664000100978007409e20002003a0000612e008f
:10665000e0030700a04b8000e10f500002003a0069
:1066600040612e00db030700a04b8000e20f5000ca
:1066700002003a0080612e00d6030700c0612e00a0
:10668000d4030700a04b80000000d000c497200076
:1066900004004000100078006101b900804f220022
:1066a0001100200037f20700809fbe0030622e00ec
:1066b000801f7800c083200021e70700e68757008d
:1066c000c0832000c3030700ab0137002d0707007c
:1066d000000f78001e00e0000200340010002000cf
:1066e000804b88001e00e00002003d000000eb002f
:1066f000804b88007009e20003003200c0622e0067
:10670000b40307009c013700d0632e00b1030700db
:10671000990137001b070700000f78001e00e000fa
:106720000200340010002000904b88001e00e000a2
:1067300002003d000000eb00904b88007209e2006f
:1067400003003200e0642e00a20307008a01370034
:10675000f0652e009f030700870137000907070037
:10676000000f78001e00e00002003400100020003e
:10677000404c88001e00e00002003d000000eb00dd
:10678000404c88008809e20003003a0000672e00b0
:10679000900307007801370010682e008d03070072
:1067a00075013700a000200000070700214c800081
:1067b00000804000204c88008409e20002003d0077
:1067c0000000eb00204c8800204c8000e30f5000bc
:1067d0000200340030002000204c880020692e0088
:1067e0007c0307008409e20002003a00b0692e0031
:1067f00078030700204c8000e10f500002003a00af
:10680000406a2e0073030700204c8000e20f500006
:1068100002003a00d06a2e006e030700204c800070
:10682000e30f500054013a00606b2e00690307002b
:1068300051013700d3060700cf80de00431c2e0035
:106840001302b800130190000283b900050178001b
:1068500006014100930178000198b9000001410050
:106860008202780020498000314980000000420007
:1068700081804a00204988003149880022498000ef
:1068800033498000f0d02c0001002000800f51001f
:10689000818f590004003400f0d02c00010020004a
:1068a000204988003149880022498000334980000e
:1068b000c07e230001002000800f5100818f59000d
:1068c00004003c00d07e2300010020002049880005
:1068d000314988002a812000204980003149800008
:1068e0004f8ade00cfa2de002049800031498000bf
:1068f0000401780084017800844c8000954c80006d
:106900004facde00cfc4de00844c8000954c80008c
:106910000803780088037800caf10700009dbe00d4
:106920000295be00208120005001be004000be0044
:10693000140220008381d1000281d3008180d30022
:106940000080d3000402e900faff3a002007980013
:106950002e0090000000d0006101b900000e270059
:1069600021072000dcf10700404988002e0090003c
:10697000801f7800f06b2e00801f7800c0832000fd
:106980006fe60700e4875700c0832000110307006b
:10699000f90037007b060700000f78001e00e000ba
:1069a0000200340010002000504c88001e00e0005f
:1069b00002003d000000eb00504c88008a09e20014
:1069c00003003200006d2e0002030700ea003700ca
:1069d000106e2e00ff020700e7003700690607006f
:1069e00080007800a00020000088b900c24b800021
:1069f00000004100c04b8800c14b8000c044200013
:106a0000808f500002003400c0442000c04b88003a
:106a10007809e20002003d000000eb00c04b880056
:106a20007809f800206f2e00801f7800c0832000b6
:106a300043e60700e4875700c0832000e502070013
:106a4000c04b800007080700cb0037004d06070049
:106a500080007800a00020000088b900b24b8000c0
:106a600000004100b04b8800b14b8000c0da20002c
:106a7000808f500002003400c0da2000b04b880044
:106a80007609e20002003d000000eb00b04b8800f8
:106a90007609f80040702e00801f7800c083200027
:106aa00027e60700e4875700c0832000c9020700db
:106ab000b04b8000f1070700af0037003106070038
:106ac00080007800d04b800001004000d04b88004f
:106ad000d14b800000e12000808f50000200340084
:106ae00000e12000d04b88007a09e20002003d005e
:106af0000000eb00d04b88007a09e20006003a0063
:106b000040712e00801f7800c08320000ce6070033
:106b10008f87e900060037007a09f80050722e00ce
:106b2000801f7800c083200005e60700e487570037
:106b3000c0832000a70207008f003700a0002000bc
:106b40001a060700314c800000804000304c88005d
:106b50008609e20002003d000000eb00304c880096
:106b6000304c8000e30f5000020034003000200061
:106b7000304c880070732e00960207008609e200f0
:106b800002003a0000742e0092020700304c800090
:106b9000e10f500002003a0090742e008d020700b1
:106ba000304c8000e20f500002003a0020752e00a9
:106bb00088020700304c8000e30f50006e003a005e
:106bc000b0752e00830207006b003700a000200084
:106bd000f6050700500f98005e0890000000e000e6
:106be0000f003200604c8000de0890000100400081
:106bf000604c88008c09e20002003d000000eb00c0
:106c0000604c8800604c8000e70f500002003400a8
:106c100070002000604c8800604c80003404070045
:106c2000614c8000800020000008b800c2232e00c4
:106c300000004100801f780040762e00801f780001
:106c4000c0832000bee50700e4875700c083200012
:106c50006002070048003700a0002000d3050700ad
:106c60008000780070498000010040007049880071
:106c700070498000e10f500002003c00200020001d
:106c80007049880070498000fa0f500002003400fb
:106c9000a00120007049880061498000704980008f
:106ca000808f5000020034007349800063498800df
:106cb00070498000e20f500006003a0010772e0065
:106cc000801f7800c08320009de507008f87e900c2
:106cd000060037002e09f80020782e00801f78006b
:106ce000c083200096e50700e4875700c08320009a
:106cf00038020700200037000040eb007500070055
:106d0000f04380000144800002ba2b00d300200031
:106d10009cf00700801f78007808f80040792e006a
:106d2000801f7800c083200085e50700e6875700b4
:106d3000c08320002702070000c4b30065000700dd
:106d4000104480002144800002ba2b00d3002000b0
:106d50008cf00700801f78007a08f800f0792e0088
:106d6000801f7800c083200075e50700e687570084
:106d7000c083200017020700344c800024179800bd
:106d80002e109000e10f50000d003200ae10900068
:106d9000e18f500004003c002e1190000200e00042
:106da000050032000a003700ae119000e28f51005a
:106db00005003200060037008d140700050037007b
:106dc000d80d0700030037002c1107000100370021
:106dd000d10a07005f120700cfc2bf000080fb008e
:106de0004600de000080fb0061006000e10f500003
:106df000fff83a00dbf707006ef70700fcf83700f2
:106e00000200fa00004f78000900fc00b116800073
:106e1000f00f2000008160001e80fb00c800dd0034
:106e200000f02f000080600000007100b0168800a4
:106e30001000200096040700d6a2a8001000200031
:106e400093040700d6a2a9001000200090040700b8
:106e50000080fa00000006000200fa00000028008e
:106e6000000f78000400fc009116800000f02f0055
:106e70000080700090168800d6c2a800d6e2a90053
:106e80001e00e0000a003d00100020008004070002
:106e9000d6a2a800200020007d040700a1168000d3
:106ea00000f02f00008f6000d6a2a900f4ff370089
:106eb000d6c2a900d6e2a8000400fc00901680000b
:106ec000f10f200001006000901688000080fa0099
:106ed000000006000200fa00004f7800deff070005
:106ee000d6e2a90000c8b3001e407000c4ff07002e
:106ef000d6e2a8000080fa00000006000000fa00b8
:106f0000d5ff0700d6e2a90010c0b300bcff070000
:106f1000d6e2a8000080fa00000006000000fa0097
:106f2000d6e2a900d6c2a900f0002000750407002f
:106f300080c3b300b2ff07005000200071040700b7
:106f400080c3b300aeff0700100020006d040700ef
:106f500080c3b300aaff07001000200069040700e7
:106f6000c0c0b300a6ff07001000200065040700a2
:106f700010c0b300a2ff070020002000610407003a
:106f800060c0b3009eff0700100020005d040700f2
:106f9000d6e2a8000080fa00000006000200fa0015
:106fa000004f7800acff07001e40780094ff0700f8
:106fb0000080fa00000006000200fa00004f78008e
:106fc00011479800a4ff0700d6e2a900f0c3b30060
:106fd0001e4f600000c4b3001e40700088ff070011
:106fe000d6e2a8009cff07001e40900084ff070027
:106ff000c2ff07000080fa00000006000400fa004b
:10700000004f7800114798000040eb00204798009f
:10701000ae4090001e40900080cf500007003d0021
:107020008dff07001e40780075ff07002e4090007e
:107030000040e80020479800f5ff37000080fa0084
:10704000000006000000fa0083ff0700d6e2a90056
:1070500000c4b3006aff0700d6e2a80011c0b30065
:107060000040eb00e5ff070051c0b30000c1b300d2
:10707000e2ff070021c0b3000040eb00dfff070084
:1070800011c0b3000040eb00dcff070051c0b300ab
:1070900040c1b300d9ff070021c0b3000040eb009e
:1070a000d6ff070011c0b3000040eb00d3ff07007c
:1070b00051c0b30050c1b300d0ff070021c0b300de
:1070c0000040eb00cdff070011c0b3000040eb0013
:1070d000caff070051c0b30010c0b300c7ff0700cc
:1070e00021c0b3000040eb00c4ff070011c0b30093
:1070f0000040eb00c1ff070051c0b30050c0b30017
:10710000beff070021c0b3000040eb00bbff07003b
:1071100021c0b3000040eb00b8ff070011c0b3006e
:1071200000c1b300b5ff070011c0b3000040eb0081
:10713000b2ff070011c0b30000c1b300afff0700ea
:1071400031c0b3000040eb00acff070031c0b3001a
:107150000040eb00a9ff070011c0b30000c1b3005d
:10716000a6ff070041c0b3000040eb00a3ff0700eb
:1071700021c0b3000040eb00a0ff070031c0b30006
:1071800000c1b3009dff070031c0b3000040eb0019
:107190009aff070059ff07000080fa000000060070
:1071a0001200fa00000f7800000320009e0f10006c
:1071b0000200340000032000000f78001e00780059
:1071c00062002000110009000200d800200798008a
:1071d0001e00780062002000110009000200d800a3
:1071e0008000fd00300798000000eb004007980089
:1071f0000000eb00100798001e009000e70f500001
:107200000e003c00ea0047004e0090000081400064
:10721000617b2e001e009000008040001049780025
:107220004e0090000000e800400798001e0090000b
:107230000000e80010079800efff37000000eb00a7
:10724000400798002e0090000000e0000c00340081
:10725000ea0047004e0090008080400020c0b3004c
:10726000804878004e0090000000e8004007980039
:107270002e0090000000e90020079800f1ff370081
:107280003e0090000000e00007003400ea004700e4
:107290004e00900000814000a17a2e003e00900038
:1072a00000804000104978000000eb0010079800b3
:1072b0001e009000e70f500009003c00ea00470064
:1072c0001e009000008040001040780033ff07004f
:1072d0001e0090000000e80010079800f4ff37003f
:1072e0000080fa00000006001600fa00000f780087
:1072f00011079800000320009e0f100002003400c8
:1073000000032000000f7800800020005007980044
:107310001e00780062002000110009000200d80061
:10732000300798001e00780062002000110009005c
:107330000200d8008000fd00400798001e00900069
:107340000000e00036003a000000eb006007980003
:107350003e0090000000e0000f003400ee00470007
:107360006e0090008080400020c0b300804878000c
:107370006e0090000000e800600798003e0090005a
:107380000000e900300798005e0090000000e9006e
:1073900050079800eeff37004e0090000000e0001c
:1073a0000d003400ee0047006e00900000814000a8
:1073b000a17a2e004e009000008040001049780015
:1073c0006e0090000000e800600798005e009000ea
:1073d0000000e900500798000000eb00200798002b
:1073e000ae0090005e009000808f500042003d0093
:1073f000ee0047006e0090008080400000c2b300a5
:10740000804878006e0090000000e8006007980057
:107410002e0090000000e80020079800f0ff3700e1
:1074200070002000600798003e0090000000e0001f
:107430000f003400ee0047006e0090008080400096
:1074400020c0b300804878006e0090000000e90082
:10745000600798003e0090000000e90030079800a7
:107460005e0090000000e90050079800eeff370032
:107470004e0090000000e0000d003400ee004700d8
:107480006e00900000814000017b2e004e009000b5
:1074900000804000104978006e0090000000e90074
:1074a000600798005e0090000000e9005007980017
:1074b0000000eb0020079800ae0090005e009000f6
:1074c000808f50000c003d00ee0047006e009000e1
:1074d0008080400000c2b300804878006e009000b9
:1074e0000000e900600798002e0090000000e8000e
:1074f00020079800f0ff37000000eb0020079800fd
:107500002e009000e70f500009003c00ee004700fd
:107510002e00900000804000104078009ffe070081
:107520002e0090000000e80020079800f4ff3700cc
:107530000080fa00000006000200fa00004f780008
:107540001e40780095fe07000080fa00000006004b
:107550000200fa00004f78001e40780010479800a3
:107560001e80fb004400de00004f780090c0b30096
:107570009e4f100003003e0000c3b3001e4f4000aa
:107580000200370070c3b3001e4f40001e40780059
:1075900082fe07001e409000004f78001e407800d9
:1075a0006f4f600090c0b3009e4f100003003e007c
:1075b00000c3b3001e4f40000200370070c3b30089
:1075c0001e4f40001e40780074fe07000080fa0045
:1075d000000006000200fa00000f78001e0078008c
:1075e0001004e000070032009e007800114078008f
:1075f0006afe07001e0078000000e800000f780017
:10760000f6ff37000080fa00000006000600fa00ce
:10761000008fbe00424798004e4090000004e000fa
:107620002e003a001e00be0002a02c00a3b92300c9
:1076300054ee07000043b00058fe07001e00be00d5
:1076400002a02c00a3b923004eee070002a02c00dc
:107650000202b800a2b923000283b9000501780034
:107660000601410003a02c000388b900000141007d
:10767000820278001e1f12001e971a00e0c2b3009b
:1076800046fe07001e00be0002102e00535f2000c1
:107690003cee07000043b00040fe07001e00be00a5
:1076a00002102e00535f200036ee070002102e005d
:1076b0000202b800525f20000283b9000501780081
:1076c0000601410003102e000388b90000014100ab
:1076d000820278001e1f12001e971a004e40900072
:1076e0000004e0000a0032001e00be00026829000b
:1076f0008309200023ee0700e00f5000e08f5800c0
:1077000003003a0000c2b30024fe07000600370061
:107710001e00be00026829008309200019ee070040
:107720000043b0001dfe07001e00be0002682900d5
:107730008309200013ee0700026829000202b80046
:10774000820920000283b90005017800060141008a
:10775000036829000388b900000141008202780013
:107760001e1f12001e971a001e00be0002242400d5
:10777000f300200003ee07000043b00007fe0700ff
:107780001e00be0002242400f3002000fded0700cf
:10779000022424000202b800f20020000283b90093
:1077a0000501780006014100032424000388b90084
:1077b00000014100820278001e1f12001e971a006d
:1077c000e0c2b300f5fd07001e00be00026a2800fb
:1077d00013002000ebed07000043b000effd0700b1
:1077e0001e00be00026a280013002000e5ed07001d
:1077f000026a28000202b800120020000283b900c9
:107800000501780006014100036a28000388b900d9
:1078100000014100820278001e1f12001e971a000c
:107820001e00be000271220003002000d5ed0700fb
:107830000043b000d9fd07001e00be000271220007
:1078400003002000cfed0700027122000202b80001
:107850000001eb000283b900050178000601410038
:10786000037122000388b900000141008202780000
:107870001e1f12001e971a001e00be00823e20002e
:1078800003002000bfed07000043b000c3fd070068
:107890001e00be00823e200003002000b9ed07005c
:1078a000823e20000202b8000001eb000283b90012
:1078b0000501780006014100833e20000388b900dd
:1078c00000014100820278001e1f12001e971a005c
:1078d000e0c2b300b1fd07001e00be00420620005a
:1078e00003002000a7ed07000043b000abfd070038
:1078f0001e00be004206200003002000a1ed07008c
:10790000420620000202b8000001eb000283b90029
:107910000501780006014100430620000388b900f4
:1079200000014100820278001e1f12001e971a00fb
:107930001e00be00a20020000300200091ed070001
:107940000043b00095fd07001e00be00a20020000d
:10795000030020008bed0700a20020000202b80007
:107960000001eb000283b900050178000601410027
:10797000a30020000388b9000001410082027800c2
:107980001e1f12001e971a004e4090000004e000d7
:1079900003003a0001c3b3001ec040007ffd070092
:1079a0000080fa00000006000400fa00008fbe000c
:1079b00012c0b3001e00be0014ff07000080fa00d2
:1079c000000006000200fa00000f78001e00e00030
:1079d00002003400b0c2b30070fd07001e00e000da
:1079e00002003a0000c2b3006cfd07001e00e00078
:1079f00003003d00d0c2b30068fd07001e0fea007f
:107a00001e007800823e2000110009000200d8000c
:107a10000043b00061fd07001e007800823e200098
:107a2000110009000200d8008000fd00803e200007
:107a30000088b9001e0f1000e0c2b30057fd070018
:107a40001e00780042062000110009000200d80044
:107a50000043b00051fd07001e00780042062000e0
:107a6000110009000200d8008000fd00400620003f
:107a70000088b9001e0f10001e007800a200200030
:107a8000110009000200d8000043b00043fd0700c8
:107a90001e007800a2002000110009000200d8009a
:107aa0008000fd00a00020000088b9001e0f10001b
:107ab0000080fa00000006000400fa00000f7800c1
:107ac00011079800f07022009e0f10000200340091
:107ad000f0702200000f78001e007800823e200027
:107ae000110009000200d8000000e0000f00320081
:107af0001e007800823e2000110009000200d8001c
:107b00000043b00025fd07001e007800823e2000e3
:107b1000110009000200d8008000fd00803e200016
:107b20000088b9001e0f10000200370000c2b30029
:107b30001afd07001e00780042062000110009000f
:107b40000200d8000043b00014fd07001e007800ba
:107b500042062000110009000200d8008000fd004c
:107b6000400620000088b9001e0f10001e00900083
:107b7000e20f5000040032009e00900070072000c9
:107b8000808f500002003a00e0c2b30003fd0700fe
:107b90001e007800a2002000110009000200d80099
:107ba0000043b000fdfc07001e007800a20020008a
:107bb000110009000200d8008000fd00a000200094
:107bc0000088b9001e0f10001e009000e10f500049
:107bd00002003a00e0c2b300f0fc07009e009000f3
:107be00070072000808f500003003a0070c5b3007a
:107bf000eafc07000300370001c3b3001ec04000c9
:107c0000e6fc07000080fa00000006000200fa000f
:107c1000004f780090c0b3009e4f10000200340067
:107c200090c0b300004f780001c3b3001ec04000f5
:107c3000dafc07000080fa0000000600809fbe000a
:107c40000400fa0090108000004f780062cdbf0061
:107c50000040e80020479800ae409000bec9bf0039
:107c6000000ce1000800320062cdbf000080fb0084
:107c7000f19b2000010040001e48780062cdbf004b
:107c80000040e80062edb7000ec2bf000080fb00bc
:107c90000000d1000080fb0061006000e10f500097
:107ca00001003a000e22a9008520a9000080fa00f8
:107cb0004f00be00004006000000fa00e07b2e00ee
:107cc00030009000a01088000000eb0060108800d9
:107cd0000000eb00701088008520a9008d20a8000e
:107ce0000de2a8000f42a8000080fa000000060084
:107cf0000200fa00000f7800700020009e0f1000b4
:107d00000200340070002000000f7800e17b2e009c
:107d10001e0078000000d000010040001000780034
:107d2000a01088000080fa00000006000200fa009f
:107d3000004f78000fc2bf000080fb000000d100a0
:107d40000080fb0061006000e10f5000f9ff32008d
:107d50001e00fb00f10f2000010060008010880071
:107d60000080fa00000006000200fa0021d6200080
:107d700091407800bec9bf0000c05000004fe9002c
:107d80001e80fb000080fa00000006000000fa00e0
:107d90000040eb00bee9b70010c0b30062edb700d1
:107da0000080fa00000006000200fa000000000057
:107db000bec9bf000040e800004f78009e40780038
:107dc00062cdbf00000ce100f9ff3200bec9bf0068
:107dd0000040e800bee9b700bec9bf000080fb005c
:107de000f19b2000010040001080fb000080fa00a1
:107df000000006000200fa00ebff0700004f7800c9
:107e00001e407800c9ff07001e80fb000080fa00ba
:107e1000000006000600fa006000b800008fbe00f7
:107e2000e1ff07000074a100404798004e40900019
:107e3000beff0700ce409000f0c2b30080cf5000dc
:107e400016003400ce40900090c3b30080cf5000a5
:107e500012003c001e00be00a20020000203b80079
:107e60000001eb000282b900070178000401410023
:107e7000a30020000388b9000001410082037800bc
:107e80004e4090000000fb0001fd2f00010040006b
:107e9000cf80de00001f430001974b004e40900052
:107ea000ed4f5000deff3a001e00be000080fa00d9
:107eb000000006000600fa00881f7800008fbe0050
:107ec00090c0b300504798000040eb004047980036
:107ed0004e409000e94f500016003c005e4090007c
:107ee0000000fb00f1ab2000010440001e00be00ba
:107ef000a20020000300200087ec070002c3b300ab
:107f0000024c40001e00be00a20020000300200022
:107f100071ec0700008fbe005e4090000040e90059
:107f2000504798004e4090000040e80040479800bd
:107f3000e7ff37000040eb00c9eab7004f047800c4
:107f40000080fa00000006000400fa00008fbe0066
:107f50001e00be00d7ff0700bfcabf0073ff0700a7
:107f6000c0cabf0071ff0700c1cabf006fff070092
:107f7000c2cabf006dff0700c3cabf006bff070086
:107f8000c4cabf0069ff0700c5cabf0067ff07007a
:107f9000c6cabf0065ff0700c7cabf0063ff07006e
:107fa000c8cabf0061ff07000080fa000000060099
:107fb0000200fa0062cdbf000080fb00801f780045
:107fc000bec9bf000080fb00801f7800e07c2e004f
:107fd000801f7800f9e00700e68757000000eb00fb
:107fe000000f7800e00f20009e0f100006003c00fc
:107ff000f19b20001e804000104078004bff0700de
:108000001e0fe800f7ff37000080fa0000000600ae
:108010000000fa000000eb0050158800f01f20005f
:1080200040158800f000200030158800000820006e
:10803000201588000000eb001015880000002800c3
:10804000001588000080fa00000006000200fa0017
:10805000000f78009e0078006f8060003015880067
:10806000a022a800401f200009000700a022a900ac
:10807000a0c2bf000080fb00610060000000e000c3
:10808000fbff3200001480000080fa0000000600b0
:108090000200fa00000f78000000eb00c008880022
:1080a0001e00780001002000820020000202b800bb
:1080b0000001eb000283b9000501780006014100d0
:1080c000830020000388b90000014100820278008b
:1080d000e408880086c0a90021e1a80086c0bf008e
:1080e0000080fb004600de000080fb0061006000b5
:1080f0000000e000f9ff320021e1a9000080fa0051
:10810000000006000400fa00000f78000000eb00f9
:10811000100798001e0090009e0f500006003100ce
:10812000803e2000daff07001e0090000000e800fb
:1081300010079800f7ff37000080fa0000000600e3
:10814000809fbe00821f78000200fa000000eb0052
:10815000000f780082c0bf000080fb004400de00fa
:108160000080fb00610060000000e00002003a00b7
:1081700011002000010f78009e40780061c060006f
:108180004401dd002108200091407800f0ceb300ca
:1081900000c060000240700082e0b70088a0a90023
:1081a00010c0b3003eedb700400de20024003200e5
:1081b00082c0bf000080fb004400de000080fb00a6
:1081c000610060000000e0000f003a00c3c2bf0081
:1081d0000080fb004600de000080fb0061006000c4
:1081e0000000e00004003200e06980000000e800c8
:1081f000e069880012003700e06980000000e900b3
:10820000e06988000e003700c3c2bf000080fb0099
:108210004600de000080fb00610060000000e0001e
:1082200004003200e06980000000e900e069880095
:1082300003003700e06980000000e800e069880082
:108240000000eb00006a88000080fa004f0178000f
:108250004f00be0000400600809fbe00821f7800d5
:108260000200fa000000eb00000f780082c0bf009f
:108270000080fb004300de000080fb006100600026
:108280000000e00002003a0011002000010f780019
:108290009e40780061c060004301dd00210820009d
:1082a0009140780070cfb30000c0600002407000c1
:1082b00082e0b7008880a90010c0b3003eedb7008f
:1082c000400de20022003a0082c0bf000080fb00a7
:1082d0004300de000080fb00610060000000e00061
:1082e0000e003a00c3c2bf000080fb004700de0062
:1082f0000080fb000000e00004003200e069800024
:108300000000e900e069880011003700e0698000a2
:108310000000e800e06988000d003700c3c2bf001c
:108320000080fb004700de000080fb000000e00052
:1083300004003200e06980000000e800e069880085
:1083400003003700e06980000000e900e069880070
:1083500010002000006a88000080fa004f017800b9
:108360004f00be00004006000000fa0088a0a900ef
:1083700090a0a8008880a9009080a8000080fa0042
:10838000000006000200fa00e0698000000f78009b
:108390000000eb00e06988000040eb003eedb70014
:1083a0001e0078000080fa00000006000600fa00b7
:1083b000000f7800e06980009e0f50000700340035
:1083c0000000eb00e06988000040eb003eedb700e4
:1083d00010002000200798000d0037009e00ea00e2
:1083e000e0698000810f500007003d000000eb00b5
:1083f000e06988000040eb003eedb7000080eb0034
:1084000020079800020037000000eb0020079800ca
:108410002e0090000080fa00000006000200fa0022
:10842000004f78000040eb00104798001e4090007d
:10843000e74f500010003c001e80fb006100600010
:108440000000e00002003200e202a8000100370054
:10845000e202a900e222a8001e80fb000000d10079
:10846000004f7800e222a9001e4090000040e80082
:1084700010479800edff37000080fa00000006006a
:108480000600fa00008fbe001e00be00106a8800c1
:10849000216a88000040eb00404798004e40900061
:1084a000e44f50000a003c004e4090000000fb00ea
:1084b00021d420000100400010407800d7ff0700c1
:1084c0004e4090000040e80040479800f3ff37001e
:1084d000e822a800e822a9000080fa0000000600b7
:1084e0000000fa00e802a800e202a900e802a900e0
:1084f000e822a800e822a90010c0b30046edb700aa
:108500000080fa00000006003200f80090018800a8
:108510006118e100040032007018e100020032002e
:10852000f0ff2f00030037003119ba008301e90082
:10853000fdff3a003200f90000000600849fbe00f3
:108540004220a900440424006110e1000a00320026
:10855000540424007010e100070032006404240079
:10856000f5ff2f000510e10003003200f0ff2f009f
:108570004f02be00000006003200f800203b8800d9
:10858000113b8800043b88000500fc0050052000da
:10859000303b8800a00a2000303b880061e7a8003b
:1085a000000000000000000061e7af00feff3700a0
:1085b0000000eb003200f9004f02be000000060090
:1085c000841f78004220a900440024006118e100c3
:1085d00006003200540024007018e100030032004d
:1085e0004f027800f0ff2f00000006003200f80074
:1085f00091018800821f78003019bb008301e900d7
:10860000fdff3a00213b88004f017800123b8800b3
:10861000043b88000500fc0050052000303b88002a
:10862000a00a2000303b880061e7a800000000009d
:108630000000000061e7af00feff37000000eb0024
:108640003200f9004f027800000006003600f80002
:10865000809fbe00829fbe00849fbe00869fbe009a
:108660000200fa0030032000a01088000000eb0098
:10867000000f7800f0cf27009e0f100003003c0091
:10868000000000001e0fe800faff3700a07e2e0059
:10869000801f780049df07008f87e9004207f80054
:1086a00040802e00801f780044df0700e4875700d9
:1086b0009a000700ffff37003600f800809fbe00d9
:1086c000829fbe00849fbe00869fbe000000fa000d
:1086d000f0658800016688001266880023668800bd
:1086e000346688004566880056668800676688009c
:1086f00078668800896688009a668800ab6688007c
:10870000bc668800cd668800de668800ef6688005b
:1087100020812e00801f780028df07008f87e90066
:10872000be0cf800a0822e00801f780023df070017
:10873000e4875700c00cf80040832e00801f7800ab
:108740001edf0700e4875700c20cf800e0832e000c
:10875000801f780019df0700e4875700c40cf80079
:1087600080842e00801f780014df0700e487570004
:10877000c60cf80020852e00801f78000fdf070050
:10878000e4875700c80cf800c0852e00801f7800d1
:108790000adf0700e4875700ca0cf80060862e0045
:1087a000801f780005df0700e4875700cc0cf80035
:1087b00000872e00801f780000df0700e487570045
:1087c000ce0cf800a0872e00801f7800fbde07008b
:1087d000e4875700d00cf80040882e00801f7800f6
:1087e000f6de0700e4875700d20cf800e0882e0080
:1087f000801f7800f1de0700e4875700d40cf800f2
:1088000090892e00801f7800ecde0700e487570077
:10881000d60cf800408a2e00801f7800e7de0700a3
:10882000e4875700d80cf800f08a2e00801f7800eb
:10883000e2de0700e4875700da0cf800a08b2e0078
:10884000801f7800ddde0700e4875700dc0cf800ad
:10885000508c2e00801f7800d8de0700e487570078
:108860002e000700ffff37003600f800809fbe0093
:10887000829fbe00849fbe00869fbe000000fa005b
:10888000ef6688000f902000008d2e00801f78007a
:10889000cade07008f87e900dc0cf800508c2e0040
:1088a000801f7800c5de0700e48757001b00070023
:1088b000ffff37003600f800809fbe00829fbe0099
:1088c000849fbe00869fbe000000fa00608e2e00ce
:1088d000801f7800b9de07008f87e9000f000700ce
:1088e000ffff37003600f800809fbe00829fbe0069
:1088f000849fbe00869fbe000000fa0090a0a900e1
:108900009120a900b08f2e00801f7800abde0700f9
:108910008f87e90001000700ffff37000000fa0021
:1089200076f9070080912e002afb0700cfc2bf0016
:108930000080fb004600de000080fb00610060005c
:10894000e10f5000f9ff3a00cfa2a900f7ff37006e
:108950000000fa001000200050678800100020007e
:1089600060678800803e2000f06688000000eb0011
:10897000800c88000000eb00b00c8800400620004e
:10898000600c880040062000700c8800e000200089
:10899000800c8800007d2000900c8800007d200065
:1089a000a00c8800e0002000b00c8800b0d42100aa
:1089b0007008880013e1a8008ce0a8000080fa008d
:1089c000000006000000fa000000eb00200c880008
:1089d000f0002000000c8800f0002000100c88003f
:1089e00060002000200c8800e00120006008880062
:1089f00011e1a8000080fa00000006000000fa0063
:108a000011e1a9000080fa00000006000000fa0051
:108a100011e1a8000080fa00000006000000fa0042
:108a2000f06680000080fa00000006000200fa00f4
:108a3000000f7800100020009e0f100002003e0082
:108a400020002000000f78001e0078000000d100f8
:108a5000000c88001e00e900600888000080fa0011
:108a6000000006000200fa00000f78001e007800e7
:108a7000600c88000080fa00000006000200fa0086
:108a8000000f78001e007800900c88000080fa002b
:108a900000000600809fbe00821f78000800fa00d8
:108aa0003067800030079800be009000e18f5000d2
:108ab0000c0032003e009000e10f50000600340030
:108ac000be009000e28f5000200032003e00900077
:108ad000e30f50003b003200d222a8008c60a900b6
:108ae0004c0037008000eb00010f7800d6c2bf00b9
:108af0000080fb000000d1000080fb0061006000ee
:108b00000000e00002003a0010002000000f780092
:108b10009e40780061c060000041d000612d2000bf
:108b200091407800d0cfb30000c0600002407000d8
:108b3000d6e2b700100880000000d10010088800bd
:108b40000000eb0030678800320037000000eb00c7
:108b500010079800d6c2bf000080fb000000d100c3
:108b60000080fb00610060000000e00002003a00ad
:108b70001100200011079800ae40900061c0600015
:108b80000041d000612d200091407800d0cfb3008b
:108b900000c0600002407000d6e2b700d6c2bf003d
:108ba0000080fb000000d1000080fb00610060003d
:108bb0000000e0001700320010002000306788003d
:108bc000140037000000eb0020079800d6c2bf0059
:108bd0000080fb000000d1000080fb00610060000d
:108be0000000e00002003a00110020002107980078
:108bf000ce40900061c060000041d000612d200097
:108c000091407800d0cfb30000c0600002407000f7
:108c1000d6e2b7008460a9000080fa004f01780016
:108c20004f00be00004006000200fa00000f78006e
:108c300030002000306788001e00e900100888001e
:108c4000100880000000d10000088800d622a9008a
:108c5000d222a90005e1a8008460a9008c60a800c8
:108c60000080fa00000006000000fa00200020004a
:108c7000306788000080fa00000006000400fa0057
:108c8000000f780011079800e20ce2000c003a0097
:108c90001e0090000000e00009003400e40ce20037
:108ca00007003a0059ff0700401f200010458800c8
:108cb0001e009000006788001e007800daff0700a1
:108cc0000080fa00000006000000fa000000eb003f
:108cd000406788003008e20006003200cae2a800bf
:108ce00081678000700020000088b90070678800ec
:108cf000ca62a8008167800040498000dfff07004a
:108d0000806780000000d000106788000080fa00b3
:108d1000000006000000fa001000200040678800f4
:108d20003008e20006003200cae2a8008167800035
:108d3000700020000088b90070678800ca62a8002f
:108d400081678000300020000088b9008000780032
:108d500040498000c9ff0700816780004000200073
:108d60000088b900106788000080fa000000060043
:108d70003600f800809fbe00829fbe00849fbe0028
:108d8000869fbe000200fa0084e0a900e00ce20029
:108d90000e003200006780000000e90000678800d4
:108da000e00ce20009003a00afff070060498000d4
:108db0000000d0000193200001004000310020009d
:108dc000908f100001003200ca62a900ee0ce20090
:108dd00006003200706780000000e90070678800bc
:108de000ee0ce20001003a00cae2a900e20ce20047
:108df0000c003200106780000000e9001067880056
:108e0000e20ce20007003a00e80ce20003003a003e
:108e1000100020005067880002003700100020007a
:108e200060678800f60ce20003003200b067800043
:108e30000000e900b0678800c0418000e20f5000e8
:108e400013003a00c8c2bf000080fb004500de00ee
:108e50000080fb00610060000000e00002003a00ba
:108e60000000eb0050678800c8c2bf000080fb0014
:108e70004400de000080fb00610060000000e000b4
:108e80001b003a000000eb00606788001800370004
:108e9000c8c2bf000080fb004500de000080fb0070
:108ea000610060000000e00003003a000000eb00f9
:108eb00050678800020037001000200050678800cb
:108ec000c8c2bf000080fb004400de000080fb0041
:108ed000610060000000e00003003a000000eb00c9
:108ee000606788000200370010002000606788007b
:108ef000c0418000000f78009e007800e28f500093
:108f000004003c001e0078000000e0001a003c0055
:108f1000030037009e007800e38f500030003200dd
:108f2000c8c2bf000080fb004500de000080fb00df
:108f3000610060000000e00004003a00e20ce20082
:108f400002003a0060ff070047003700c8c2bf00b8
:108f50000080fb004400de000080fb006100600038
:108f60000000e00040003a00e20ce2003e003a005f
:108f700068ff07003c003700e80ce2000c003200fc
:108f8000ea0ce20004003a00e20ce20002003a00bf
:108f90004dff070034003700ec0ce20032003a00cd
:108fa000e20ce20030003a005aff07002e003700c2
:108fb000ec0ce20004003a00e20ce20002003a008d
:108fc00054ff070028003700ea0ce20026003a00b0
:108fd000e20ce20024003a003bff070022003700c9
:108fe000c8c2bf000080fb004500de000080fb001f
:108ff000610060000000e0000e003a00e40ce200b6
:1090000004003a00100020002067880040498000da
:1090100005ff07003008e20006003200cae2a8009f
:1090200081678000700020000088b90070678800a8
:10903000ca62a800c8c2bf000080fb004500de0075
:109040000080fb00610060000000e00006003200cc
:10905000e40ce20004003200ca62a90002ff07002b
:109060000000eb0020678800f06680000000e90047
:10907000f0668800de0ce2000e003a00803e200020
:10908000f0668800b04180000000e800b041880030
:10909000a608e20007003200304580000000e90029
:1090a00030458800a608e20002003a0010002000c7
:1090b00040458800a208e20003003200104580000d
:1090c0000000e90010458800f20ce20003003400c3
:1090d000906780000000e90090678800f40ce200cf
:1090e00003003200a06780000000e900a06788004c
:1090f0000080fa004f03be004f02be004f01be00c9
:109100004f00be003600f900004006000000fa00e3
:10911000ca42a9000000eb00506a88000000eb0082
:10912000606a880090432000101188000000280029
:10913000001188008500a9008d00a8000080fa00b9
:10914000000006000200fa00000f7800606a80004c
:109150009e0f10000b00320020c2bf000080fb00f9
:109160000000d1000080fb00610060000000e00012
:10917000f9ff3a001e007800201188001e007800d8
:10918000606a88000080fa0000000600801f7800f6
:109190000200fa00ca42a8008500a90020c2bf0050
:1091a0000080fb00610060000000e000040032006d
:1091b00020118000406a880010002000506a88005a
:1091c000ca42a9000080fa004f0078000040060063
:1091d0001c00fa000000eb0060498800300020000d
:1091e000804988000000eb00000f780043f707007b
:1091f000a0922e00801f780070dc07008f87e900a6
:1092000070942e00801f78006cdc07008f87e900c7
:10921000c8c2bf000080fb004600de000080fb00eb
:10922000610060000000e000040032001000200037
:10923000a0418800ca62a900030037000000eb00cb
:10924000a0418800ca62a800d00020007ffb070070
:10925000c0438800c00020007cfb0700d04388008a
:10926000c1438000c04380000088b900f0438800fb
:1092700001448800d1438000d04380000088b900b9
:109280001044880021448800f24380000344800099
:10929000104480002144800000005100818059006a
:1092a000304488004144880086ed0700c3c2bf00f7
:1092b0000080fb004500de000080fb0061006000d4
:1092c0000000e00013003a001e0fe80060002000dc
:1092d0009e0f1000020034000000eb00000f780029
:1092e00021032000e055220064fe0700c3c2bf0036
:1092f0000080fb004500de000080fb006100600094
:109300000000e000f9ff3200400620007dfb07006e
:109310001cfc07001e017800520f9800de09900027
:10932000e38f51009f0032005e089000e30f500071
:1093300007003c005e099000e10f51002700320059
:10934000de099000e18f51006f003c0009003700fa
:109350005e089000e50f5000c90032005e099000e1
:10936000e40f5100aa003400de099000e68f51009e
:10937000de0032000040eb00d6f60700e0972e003a
:1093800094f8070000c4b300d2f60700fdfb070005
:10939000cf80de00824c8000934c800002014000b0
:1093a00083814800824c8800934c8800e600470087
:1093b000824c8000934c8000829fbe00f0982e006b
:1093c000801f780001007800dddb0700e68757008a
:1093d000660047007ff80700cc0037000040eb0034
:1093e000bcf60700a000200018fb0700cf80de00bd
:1093f000c24c80000202b800d24c80000283b90047
:109400000501780006014100c34c80000198b900b5
:109410000001410082027800140798002507980097
:109420001e009000ae009000c809dd004800de007c
:1094300000807100c808de0080438800a0992e00db
:1094400064f8070021002000804380009af907009b
:10945000309a2e005ff8070000c4b3009df60700a5
:1094600050002000d1fb0700cf80de00c24c8000fe
:10947000d34c80000201400083814800c24c880028
:10948000d34c8800c24c8000d34c800030062000b2
:1094900001002000800f5100818f590004003c0022
:1094a0004006200001002000c04c8800d14c8800fc
:1094b000c24c8000d34c8000800c200001002000b2
:1094c000800f5100818f590004003400800c20006f
:1094d00001002000c04c8800d14c88006600470085
:1094e000c24c8000d34c8000829fbe00719a2e0037
:1094f000811f780092db0700e6875700660047006f
:1095000034f80700810037000040eb0071f60700d7
:10951000e6004700a09b2e00801f78000100780025
:1095200087db07008f87e9006600470029f80700fe
:1095300000c4b30067f60700500020009bfb070043
:1095400080007800500020000088b900424d800063
:1095500000004100404d8800a809e20002003d00e3
:109560000000eb00404d8800414d80004006200087
:10957000808f50000200340040062000404d8800db
:1095800066004700a809f800b19c2e00811f7800f2
:109590006bdb0700e4875700660047000df8070003
:1095a0005a0037000040eb004af6070035ec070090
:1095b000c09d2e0007f8070000c4b30045f6070061
:1095c00070fb0700cf80de00e24c8000f34c80008f
:1095d0000201400083814800e24c8800f34c88007f
:1095e000e6004700e24c8000f34c8000829fbe0002
:1095f000409e2e00801f78000100780050db07009d
:10960000e687570066004700f2f707003f00370083
:109610000040eb002ff60700509f2e00edf70700eb
:1096200042ec070000c4b3002af6070050002000f7
:109630005efb0700cf80de00224d8000334d8000ae
:109640000201400083814800224d8800334d88008c
:10965000e6004700224d8000334d8000829fbe000f
:10966000709a2e00801f78000100780034db07001c
:10967000e687570066004700d6f70700230037004b
:109680000040eb0013f60700e09f2e00d1f7070023
:1096900057ec070000c4b3000ef6070039fb0700c3
:1096a000cf80de00a24c8000b34c8000020140005d
:1096b00083814800a24c8800b34c8800e600470034
:1096c000a24c8000b34c8000829fbe00409e2e00c2
:1096d000801f78000100780019db0700e68757003b
:1096e00066004700bbf70700080037000040eb00aa
:1096f000f8f5070070a02e00b6f7070000c4b3000d
:10970000f4f5070080a12e00b2f7070063002000e7
:109710009e8f11002e003a00c3c2bf000080fb00e4
:109720004400de000080fb00610060000000e000fb
:1097300043003a00803e2000b0678800c3c2bf00eb
:109740000080fb004400de000080fb006100600040
:109750000000e0003a003a00f60ce200f7ff3a00a1
:1097600033ea070036eb0700d9ea0700414d8000d5
:10977000a00020000088b90080007800c0f6210019
:109780003efd07000000eb0050438800dbf50700ba
:1097900090a22e008ff70700a0a32e00801f780054
:1097a00006db07008f87e900c05d200055fa07003f
:1097b000c3c2bf000080fb004400de000080fb004d
:1097c000610060000000e000f9ff32002500370072
:1097d000c3c2bf000080fb004400de000080fb002d
:1097e000610060000000e00015003a0014eb070083
:1097f000414d8000c0f6210020fd07000000eb0075
:1098000050438800bdf5070060a52e0071f70700e2
:1098100040a62e00801f7800e8da07008f87e90055
:10982000c3c2bf000080fb004400de000080fb00dc
:10983000610060000000e000f9ff3200090037001d
:10984000cfc2bf000080fb004600de000080fb00ae
:1098500061006000e10f50006dfe3a00d5ec07009a
:109860006bfe37000080fa00000006000600fa00d8
:10987000c0a82e00801f7800d0da07008f87e9008b
:109880000000eb00000f7800f01f20009e0f10007a
:1098900019003c006401470000002f009e004000ba
:1098a00013002000f007200017fb070010079800a6
:1098b0001e0078006f0060000000e00006003a0023
:1098c0001e007800801f780030aa2e00801f7800cc
:1098d000bada0700e48757002e009000801f780056
:1098e000b0aa2e00801f7800b4da0700e487570082
:1098f0001e8fe800e4ff37001e009000801f7800f4
:1099000000ab2e00801f7800acda0700e487570018
:109910000080fa00000006001000fa0012f90700ab
:109920000000e000ea0132001ff90700204f980014
:109930002e4890000081fb0003002000f0fd2f0066
:10994000f1ff2f0002014000838148006207980068
:109950007307980030052000010020006e01900080
:10996000fe019000800f5100818f5900cd013e0013
:109970006e009000fe0090000060010006013700bc
:10998000c8013700c7013700c6013700c5013700dd
:10999000c4013700c3013700c2013700c1013700dd
:1099a000c00137004e013700be01370062013700a9
:1099b000bc013700bb0137007c0137009b01370039
:1099c0009a01370099013700980137009701370055
:1099d00096013700b3013700b20137008301370029
:1099e000b0013700af013700ae013700ad013700dd
:1099f000ac013700ab013700aa0137004400370043
:109a0000a801370054003700f1003700500037003c
:109a1000a4013700a3013700a20137002b00370053
:109a2000a00137009f0137009e0137009d013700dc
:109a30009c0137009b0137009a01370099013700dc
:109a4000980137009d0037009601370095013700d7
:109a5000940137005100370092013700910137001f
:109a6000840137008f0137008e0137008d013700e8
:109a70008c0137008b0137008a01370089013700dc
:109a80005d003700070137009a0037008501370075
:109a90003f01370083013700820137008101370021
:109aa000800137007f0137007e013700ef0037006b
:109ab0007c013700e5003700870037007901370067
:109ac0007801370076003700ef003700a0ac2e0099
:109ad000801f780039da07008f87e90010af2e0069
:109ae000801f780035da07008f87e900a0192e0063
:109af000801f780031da07008f87e90050b02e0010
:109b0000801f78002dda07008f87e9007001370089
:109b100090002000000f7800f10020009e8f1000c0
:109b20006b013c001e00780048f90700801f780098
:109b30001e017800821f7800a0b22e00801f7800de
:109b40001eda0700e68757001e0fe800f2ff370015
:109b500046ff07005e01370080b32e00801f7800ab
:109b600016da07008f87e9000000eb002007980055
:109b700012002000e11f2f00f00720006ffa0700fd
:109b80006400470013002000e21f2f00f1072000af
:109b90008bfa070035ff07004d01370070b52e0026
:109ba000801f780005da07008f87e9002e489000b3
:109bb000fb4f5000460132006bf807000000e00048
:109bc000fdff320078f80700204f98002e489000e3
:109bd0000080fb00801f780030b62e00801f7800c8
:109be000f6d90700e48757002e4890000080fb005c
:109bf00051f60700edff3700f0b62e00801f780009
:109c0000eed907008f87e9000040eb00204f980055
:109c1000baf407000000eb00000f7800f005200008
:109c20009e0f100008003c000040eb00a9f4070064
:109c30001e0078005af507002003200031f90700c4
:109c40001e0fe800f5ff370000c4b300a1f40700c1
:109c50002e4890000080fb00801f78002e48900066
:109c60000080fb00801f780000b92e00801f780064
:109c7000c0832000b2d90700e6875700c0832000c8
:109c800054f607002e4890000040e800204f98004e
:109c900035f807000000e000deff32000c0137005d
:109ca000c0b92e00801f7800c4d907008f87e90053
:109cb00010002000704388000501370030ba2e00e4
:109cc000801f7800bdd907008f87e9000000eb00f6
:109cd00070438800fe003700a008f8007608f800fe
:109ce000e0ba2e00801f7800b4d90700e68757003d
:109cf000f70037002c09f80080bc2e00801f780088
:109d0000aed90700e48757002208f80060be2e0095
:109d1000801f7800a9d90700e48757001041800010
:109d20000000d000039320000300400010007800e2
:109d3000801f780060bf2e00801f78009fd9070029
:109d4000e48757003409f800a0c12e00801f780076
:109d50009ad90700e48757003008f80080c32e0026
:109d6000801f780095d90700e48757003208f80073
:109d7000a0c42e00801f780090d90700e487570008
:109d80003408f800a0c52e00801f78008bd907008a
:109d9000e4875700ce00370090c62e00801f780061
:109da00086d907008f87e900fff70700204f98004a
:109db0002e489000ddf707002e4890000080fb0041
:109dc00001fd2f0001004000a0498800c0003700bd
:109dd0004af407000040eb00204f98002e48900006
:109de000fb4f5000ba003200dff707000000e00030
:109df00009003200ecf70700204f98002e48900031
:109e00000e0607000040eb0032f407002e489000d9
:109e10000080fb00c8f50700230607000000e000f3
:109e2000eeff320030060700204f98002e489000c9
:109e3000bef7070000c4b30026f407002e489000c8
:109e40000080fb00bcf50700e4ff3700824c800077
:109e5000934c8000829fbe0090c82e00801f780027
:109e600056d90700e687570099003700ebfa07003c
:109e7000801f7800f0c92e00801f78004fd907009e
:109e8000e48757009200370030cb2e00801f780007
:109e90004ad907008f87e90010502500a9fc070068
:109ea0008b003700c0cb2e00801f780043d90700fd
:109eb0008f87e9003e0090000000e800300798001e
:109ec0003e0090009ffc0700a00020008df80700d6
:109ed000a5f707000000e000f6ff32007c00370025
:109ee00060418000a39a2000030040001048e80071
:109ef00060418000a29a2000820040006041800002
:109f0000a39a20000300400010407800e34860005e
:109f100060418000a19a2000010040001080fb00f9
:109f2000801f7800a0cc2e00801f780023d9070066
:109f3000e48757006600370060418000a29a200045
:109f4000020040001048e90060418000a39a200010
:109f50008300400060418000a29a2000020040007f
:109f600010407800e348600060418000a39a200020
:109f7000030040001080fb00801f7800a0cc2e0062
:109f8000801f78000dd90700e48757005000370084
:109f9000bc09f8002c08f80010ce2e00801f7800b5
:109fa00006d90700e6875700490037000a08e20093
:109fb00007003a00e0d02e00801f7800ffd807008d
:109fc0008f87e900100020005040880040003700d3
:109fd00010d22e00801f7800f8d807008f87e90084
:109fe0000000eb0050408800390037000e08e20006
:109ff00007003a0050d32e00801f7800efd80700ea
:10a000008f87e90010002000704088003000370082
:10a01000f0d42e00801f7800e8d807008f87e90071
:10a020000000eb0070408800290037002e489000a7
:10a030000080fb006f0060000000e90060408800c5
:10a04000c21a2e0061408000400020000008b800c5
:10a05000000041001001be00829fbe000c08f80005
:10a06000a0d62e00801f7800d4d80700e8875700bc
:10a070001700370070d82e00801f7800cfd8070057
:10a080008f87e9000000eb00000f78002e009000a1
:10a090001e017800110009000200d8002007980076
:10a0a0000b0037002e4890000080fb00801f7800d6
:10a0b00050d92e00801f7800c0d80700e4875700d1
:10a0c00020da2e00801f7800bcd807008f87e900b7
:10a0d0000080fa00000006000c00fa00881f7800db
:10a0e00000b0260051542f00824c8000934c800019
:10a0f000001f4100019749001e00be008295230009
:10a100000201b800000278008402d0000302780047
:10a1100005024200859523000588b900000242002f
:10a120008401780022079800330798004f98de00da
:10a13000cf80de0040079800500798002e00900066
:10a14000be0090004e019000de01900084002000cf
:10a150008381d1000281d3008180d3000080d300ad
:10a160000402e900faff3a0020079800310798003e
:10a17000420798005307980028d1200014ee2d00c4
:10a1800055c62d0076012000070020002e0090000b
:10a19000be0090004e019000de01900000005200d1
:10a1a00081805a0002015b0083815b00009cbe003d
:10a1b0000294be004f0478000080fa000000060000
:10a1c0000c00fa000040eb0028edb70024cdbf00e2
:10a1d0000080fb004400de000080fb000100200046
:10a1e000008fbe001e00be00a20020000203b800c7
:10a1f0000001eb000282b900070178000401410070
:10a20000a30020000388b900000141008203780008
:10a2100024cdbf000080fb00010020006f00600023
:10a220008000eb00001f430001974b001e00be00a2
:10a23000a20020000203b8000001eb000282b90076
:10a240000701780004014100a30020000388b90041
:10a25000000141008203780025cdbf000080fb0093
:10a260004400de000080fb0001002000001f4300ce
:10a2700001974b001e00be00a20020000203b800a0
:10a280000001eb000282b9000701780004014100df
:10a29000a30020000388b900000141008203780078
:10a2a00025cdbf000080fb00010020006f00600092
:10a2b0008000eb00001f430001974b001e00be0012
:10a2c000a20020000203b8000001eb000282b900e6
:10a2d0000701780004014100a30020000388b900b1
:10a2e000000141008203780026cdbf000080fb0002
:10a2f0004400de000080fb0001002000001f43003e
:10a3000001974b001e00be00a20020000203b8000f
:10a310000001eb000282b90007017800040141004e
:10a32000a30020000388b9000001410082037800e7
:10a3300026cdbf000080fb00010020006f00600000
:10a340008000eb00001f430001974b001e00be0081
:10a35000a20020000203b8000001eb000282b90055
:10a360000701780004014100a30020000388b90020
:10a37000000141008203780027cdbf000080fb0070
:10a380004400de000080fb0001002000001f4300ad
:10a3900001974b001e00be00a20020000203b8007f
:10a3a0000001eb000282b9000701780004014100be
:10a3b000a30020000388b900000141008203780057
:10a3c00027cdbf000080fb00010020006f0060006f
:10a3d0008000eb00001f430001974b001e00be00f1
:10a3e000a20020000202b8000001eb000283b900c5
:10a3f0000501780006014100a30020000388b90090
:10a400000001410082027800048fbe00500020004d
:10a41000010020001e0f40005e97480000a02500ac
:10a4200021262000be0f1000ae8f1800030036005a
:10a4300000a0250021262000008fbe001e00be00c7
:10a440000001eb008001eb0024d120005403be008a
:10a450004402be00fbe20700200798003107980085
:10a4600042079800530798001141800040002000e7
:10a470000008b800c28a2000020240002e009000ae
:10a48000be0090004e019000de019000f50120001a
:10a490008381d1000281d3008180d3000080d3006a
:10a4a0008502e900faff3a00008abe000080fa0047
:10a4b000000006000200fa000000eb00000f780028
:10a4c000400020009e0f100006003c00c0d120007c
:10a4d0009e0040000040eb00804878001e0fe8001e
:10a4e000f7ff37000080fa00000006000200fa00c3
:10a4f0000000eb00000f7800400020009e0f1000cd
:10a5000006003c00c1d120001e80400010407800b1
:10a5100006f607001e0fe800f7ff37000080fa007c
:10a52000000006001400fa00889fbe00284de200db
:10a530000400320090678000e10f400001003a0003
:10a540001fff0700f20ce20005003a000000eb00dc
:10a5500010698800d7ff07000080eb009067880033
:10a5600001f607000000e000eb013200800c200043
:10a5700090678800220de20002003d000000eb0021
:10a580001069880010698000e40f50000200340058
:10a59000400020001069880010698000c1d12000af
:10a5a0000104400000f60700004c780010698000ac
:10a5b0000000e8001069880010698000e40f500076
:10a5c000d50134000000eb001069880020cdbf00e9
:10a5d0000080fb00100f9800000820001e0990006a
:10a5e000800f5100c3013200000820001e0a9000b5
:10a5f000800f52001b003c001e089000e20f50002c
:10a60000690132009e089000e28f500007003c0074
:10a610001e0990000200e000b10132001e0a900005
:10a62000e10f520093013200300037001e08900005
:10a63000e70f50007e0132009e089000e78f500027
:10a6400004003c001e099000e30f51002b00320073
:10a65000260037001e0a9000e80f520098013200d1
:10a6600022003700800820009e089000808f500054
:10a6700097013200800820001e099000800f5100d1
:10a6800009003c00100820001e0a9000800f5200b4
:10a690005a013200200820009e089000808f500050
:10a6a0004b01320011003700700e20001e0990008f
:10a6b000800f5100fc003200700e20001e0a900036
:10a6c000800f520005003c00b00b20009e08900057
:10a6d000808f50008c01320004003700700f200082
:10a6e0001e099000800f51000801320071ff070021
:10a6f00000cfb3008df50700870137006dff07001d
:10a70000d0408000e14080004f8ade00cfa2de0012
:10a71000d0408000e140800004017800840178008e
:10a72000844c8000954c80004facde00cfc4de002e
:10a73000844c8000954c80000803780088037800e2
:10a7400040e2070040079800510798006207980010
:10a75000730798004e009000de0090006e0190009c
:10a76000fe019000140220008381d1000281d300f9
:10a770008180d3000080d3000402e900faff3a0090
:10a7800020079800310798000040eb001cedb7004f
:10a790001ccdbf004404dd002e009000be009000e0
:10a7a00002682900830920004be2070000404400b2
:10a7b0001cedb7002e009000be009000026829003a
:10a7c0008309200044e20700026829000202b80061
:10a7d000820920000283b9000501780006014100ca
:10a7e000036829000388b900000141008202780053
:10a7f0002e009000be00900004005000858058009c
:10a8000020079800310798002e009000be009000ad
:10a8100002242400f30020002fe207001dedb70002
:10a820002e009000be00900002242400f3002000bf
:10a8300029e20700022424000202b800f2002000ee
:10a840000283b900050178000601410003242400b9
:10a850000388b90000014100820278002e009000b8
:10a86000be0090000400500085805800200798002a
:10a87000310798001dcdbf004404dd002e0090007c
:10a88000be009000026a28001300200012e20700b8
:10a89000004044001dedb7002e009000be00900067
:10a8a000026a2800130020000be20700026a280059
:10a8b0000202b800120020000283b90005017800ee
:10a8c00006014100036a28000388b9000001410025
:10a8d000820278002e009000be009000040050001c
:10a8e0008580580020079800310798002e009000be
:10a8f000be0090000271220003002000f6e1070074
:10a900001eedb7002e009000be00900002712200e4
:10a9100003002000f0e10700027122000202b800eb
:10a920000001eb000283b900050178000601410037
:10a93000037122000388b9000001410082027800ff
:10a940002e009000be00900004005000858058004a
:10a9500020079800310798001ecdbf004404dd0099
:10a960002e009000be009000823e200003002000d8
:10a97000d9e10700004044001eedb7002e00900012
:10a98000be009000823e200003002000d2e10700bc
:10a99000823e20000202b8000001eb000283b900f1
:10a9a0000501780006014100833e20000388b900bc
:10a9b00000014100820278002e009000be0090004d
:10a9c0000400500085805800200798003107980047
:10a9d0002e009000be0090004206200003002000e0
:10a9e000bde107001fedb7002e009000be009000f3
:10a9f0004206200003002000b7e1070042062000c5
:10aa00000202b8000001eb000283b90005017800e2
:10aa100006014100430620000388b90000014100ff
:10aa2000820278002e009000be00900004005000ca
:10aa30008580580020079800310798001fcdbf007f
:10aa40004404dd002e009000be009000a200200013
:10aa500003002000a0e10700004044001fedb70004
:10aa6000104180000000d000019320000100400050
:10aa700022002000900f110007003c0010418000d0
:10aa80000000d00004932000040040001040780033
:10aa900020edb700020037000040eb0020edb700ca
:10aaa00092fe07009c00370082fe07003408e20097
:10aab00011003200b0438000320020001100090074
:10aac0000200d800005798000e509000ef4f500041
:10aad00002003600f0c0b30000579800a408e2005e
:10aae000070032000e50900001c8b3000140700012
:10aaf000005798000200370000c0eb000057980094
:10ab00000e50900089f407008300370069fe0700ab
:10ab10003408e2001f003a00f044800032002000b8
:10ab2000110009000200d800005798000e50900054
:10ab3000ef4f500002003600f0c0b30000579800fd
:10ab40000e50900001c8b3000140700000579800fb
:10ab50009a08e200040032000e50900001c4b300d5
:10ab6000014070000057980060498000e20f5000db
:10ab70000a003a0070498000e20f500007003a00d6
:10ab80000e50900001c2b3000140700000579800c1
:10ab90000200370000c0eb00005798000e509000f4
:10aba00062f407005c00370060498000d0688800cc
:10abb00070498000e20f500002003a00200020009f
:10abc000604988000040eb0058f40700520037004d
:10abd000d0688000e10f500003003c00d168800085
:10abe00061498800020037000000eb0060498800de
:10abf0000040eb004df4070047003700704980002b
:10ac0000e20f500007003a002c09e2000300320076
:10ac10000000eb00604988000200370010002000af
:10ac2000604988000040eb0040f407003a0037001c
:10ac3000c0d1200022c0b300904f11000a003e0096
:10ac4000104180000000d0000493200084004000e8
:10ac50001ccdbf000080fb00800878000040eb00a6
:10ac600032f407002c00370000cfb3002ff40700a8
:10ac7000290037000000eb00000f780040002000a2
:10ac80009e0f10000b003c0042d220009e004100ad
:10ac9000c4d120001e00420090487800c0d120009e
:10aca0009e0040000040eb00804878001e0fe80046
:10acb000f2ff37000040eb001cf4070016003700dd
:10acc000cae2a8000040eb0018f4070012003700a9
:10acd000cae2a9000040eb0014f407000e003700a0
:10ace00010002000604388000040eb000ff40700d4
:10acf000090037000000eb00604388000040eb00d3
:10ad00000af40700040037000040eb0007f40700d6
:10ad10000040eb0005f407004f04be000080fa007d
:10ad2000000006000200fa000000eb00000f7800af
:10ad3000304c8000e20f500005003a000af4070092
:10ad40000000e0000200320010002000000f780038
:10ad5000550207000000e000020032001000200051
:10ad6000000f78001e0078000080fa000000060046
:10ad70000000fa00e922a800e8c2a800e902a90040
:10ad80000080fa00000006000600fa00000f7800bc
:10ad90000000eb00100798001e009000ef0f50001d
:10ada0001d003c00e8c2a9009e00780061806000a0
:10adb0000000e00002003200e902a80001003700b4
:10adc000e902a9001e0078000000d100000f780001
:10add0002e0090000000d10020079800e6c2bf00be
:10ade0000080fb004700de000080fb000000e00068
:10adf000040032002e0090000100280001007000c5
:10ae000020079800e8c2a8001e0090000000e8009b
:10ae100010079800e0ff37002e0090000080fa0035
:10ae2000000006000400fa00000f7800e922a900e3
:10ae30001e007800d4ff070010079800e922a80040
:10ae4000e902a9001e0090000080fa000000060040
:10ae50000600fa00000f780011079800e922a90007
:10ae60001e007800c8ff07001e009000c6ff070004
:10ae700020079800e922a800e902a9002e0090000e
:10ae80000080fa00000006000a00fa00000f7800b7
:10ae90001107980022079800e922a9001e007800f7
:10aea000b9ff0700300798001e009000b6ff0700aa
:10aeb000300798002e009000b3ff0700300798007d
:10aec000e902a9000000eb00400798004e00900046
:10aed000e70f50000a003c00e8c2a9000000000093
:10aee00000000000e8c2a800000000000000000010
:10aef0004e0090000000e80040079800f3ff370084
:10af0000e922a800e902a9003e0090000080fa00b2
:10af1000000006000200fa00e9c2a80094ff070042
:10af200010002000bfff0700d1002000508628003d
:10af3000c7ff07008000eb0090002000c4ff07005f
:10af400080007800f00f2000008f60000000eb0010
:10af5000d0418800000e20009e0f100009003a002a
:10af6000d100200050862800b9ff070000de2e0027
:10af7000801f780011d507008f87e900100020009e
:10af8000d04188000080fa00000006000200fa00ac
:10af9000000f780082db2e009e0078004000200029
:10afa0000008b8000000410010007800a06a880086
:10afb00082db2e009e007800400020000008b800d0
:10afc000000041000080e80010007800b06a8800ae
:10afd0000080fa00000006000400fa00000f78006c
:10afe000110798000000eb00b0418800c3ef070094
:10aff0001e0090000000e00008003a001e007800eb
:10b00000801f780040e12e00801f7800c083200060
:10b01000cbd40700e48757000a0037007bf607000f
:10b02000401f2000104588001e007800801f780017
:10b0300040e22e00801f7800c0832000c0d40700ab
:10b04000e4875700c083200062f10700d100200090
:10b0500050862c007eff07001e007800cbff070003
:10b06000400020006fff0700b26a8000a16a8000e4
:10b070000009200084ff0700e7c2bf000080fb003a
:10b080004400de000080fb00610060000000e00082
:10b09000180032001e0090000000e00006003200a0
:10b0a00080c0b3008bef0700d0002000e7f307005b
:10b0b000c043880095e5070000c4b30085ef070092
:10b0c0003608f800e0e22e00801f7800c0832000e0
:10b0d0009bd40700e4875700c08320003df10700a0
:10b0e00010ff07000000e000e3ff32002001200015
:10b0f0004cff0700d10020005086280054ff0700b5
:10b100000080fa00000006000400fa00000f78003a
:10b11000110798000000eb00b041880077ef0700ae
:10b120001e0090000000e0000b003a001e007800b6
:10b13000801f7800e0e32e00801f7800c08320008d
:10b140007fd40700e4875700d100200050062c0070
:10b150003fff07000d0037002cf60700401f2000be
:10b16000104588001e007800801f780010e52e0032
:10b17000801f7800c083200071d40700e487570047
:10b18000d10020005086280031ff0700c083200036
:10b1900010f1070000c4b3004eef07001e00780056
:10b1a0007aff0700400020001eff0700b26a8000ff
:10b1b000a16a80002009200033ff0700e7c2bf001a
:10b1c0000080fb004400de000080fb0061006000a6
:10b1d0000000e000f9ff3a004000200011ff0700e6
:10b1e000b26a8000a16a80001009200026ff0700d3
:10b1f000e7c2bf000080fb004400de000080fb00cf
:10b20000610060000000e000150032001e009000a8
:10b210000000e0000300320080c0b3002def070003
:10b220003ae5070000c4b3002aef07003608f8002b
:10b23000e0e22e00801f7800c083200040d4070089
:10b24000e4875700c0832000e2f00700b5fe070046
:10b250000000e000e6ff320020012000f1fe0700c0
:10b2600040002000effe0700d1002000508628009b
:10b27000f7fe07000080fa00000006000800fa0050
:10b28000b9f207000000e000ae003200c6f207008d
:10b29000204798003a08e20002003a000040eb0024
:10b2a000204798002e4090000080fb003007980057
:10b2b000d0042000be009000808f50002a00320091
:10b2c000d0042000be009000808f500011003c0090
:10b2d00090032000be009000808f500008003c00ca
:10b2e00000032000be009000808f500043003d000e
:10b2f0003e0090000000e000890032008d00370021
:10b3000050042000be009000808f50002c003200be
:10b310008800370020052000be009000808f50007c
:10b320001100320020052000be009000808f5000e8
:10b3300005003c0000052000be009000808f5000fa
:10b34000090032007b00370030052000be0090006d
:10b35000808f50001000320040052000be00900099
:10b36000808f500073003a002e4090005aedb700d5
:10b37000414d8000108f210040f60700c0e52e00ef
:10b38000801f78000dd407008f87e9002e409000c1
:10b3900066f207006b003700f0e62e00801f780091
:10b3a00006d407008f87e900200120009dfe0700da
:10b3b000414d8000108f210030f6070061003700fa
:10b3c000a0e82e00801f7800fcd307008f87e900db
:10b3d000414d8000a00020000088b9008000780066
:10b3e000108f210025f60700300520008dfe070094
:10b3f0000040eb005aedb700520037002e4090009d
:10b400000080fb0001fd2f0001004000c06a8800a1
:10b41000580df80030ea2e00801f7800e7d30700af
:10b42000e4875700c06a8000d8fe07005acdbf00ed
:10b430000080fb002007980000052000ae0090006f
:10b44000808f50001200320000052000ae009000f6
:10b45000808f500005003c00d0042000ae0090001a
:10b46000808f500026003200360037002005200073
:10b47000ae009000808f500019003200400520007f
:10b48000ae009000808f5000090032002d00370080
:10b49000e0ea2e00801f7800c8d307008f87e900fc
:10b4a0008000eb00c06a8000cbfe0700250037005b
:10b4b00000ec2e00801f7800c0d307008f87e900c2
:10b4c000e9e2a800cae2a80011002000c06a8000da
:10b4d000c1fe0700cae2a900e9e2a900190037008d
:10b4e00090ec2e00801f7800b4d307008f87e9000e
:10b4f00011002000c06a800003ff07001100370020
:10b5000010ed2e00801f7800acd307008f87e90074
:10b510008000eb00c06a8000fbfe070009003700d6
:10b5200070ee2e00801f7800a4d307008f87e900fb
:10b5300004003700b0f02e00801f78009fd3070072
:10b540008f87e9000080fa0000000600809fbe009f
:10b550000400fa00e0108000004f780064cdbf00c6
:10b560000040e80020479800ae409000cacabf00e3
:10b57000000ce1000800320064cdbf000080fb0039
:10b58000b1ac2000010040001e48780064cdbf002f
:10b590000040e80064edb70018c2bf000080fb0067
:10b5a0000000d1000080fb0061006000e10f50004e
:10b5b00001003a001822a9008700a9000080fa00c3
:10b5c0004f00be00004006000000fa00e0f02e0030
:10b5d00030009000f01088000000eb00b0108800f0
:10b5e00000402000c01088008700a9008f00a8003c
:10b5f00017e2a8001942a8000080fa000000060027
:10b600000200fa00000f7800700020009e0f10006a
:10b610000200340070002000000f7800e1f02e00de
:10b620001e0078000000d0000100400010007800eb
:10b63000f01088000080fa00000006000200fa0006
:10b64000004f780019c2bf000080fb000000d1004d
:10b650000080fb0061006000e10f5000f9ff320044
:10b660001e00fb00f10f200001006000d0108800d8
:10b670000080fa00000006000200fa00000f7800c7
:10b680001e0078001004e000050032001e00780063
:10b6900010407800e9ff07001e0fe800f8ff3700b0
:10b6a0000080fa00000006000200fa0041d62000e7
:10b6b00091407800cacabf0000c05000004fe900a6
:10b6c0001e80fb000080fa00000006000000fa0067
:10b6d0000040eb00caeab70010c0b30064edb70049
:10b6e0000080fa00000006000200fa0000000000de
:10b6f000cacabf000040e800004f78009e407800b2
:10b7000064cdbf00000ce100f9ff3200cacabf00df
:10b710000040e800caeab700cacabf000080fb00c8
:10b72000b1ac2000010040001080fb000080fa0056
:10b73000000006000200fa00ebff0700004f78004f
:10b740001e407800bdff07001e80fb000080fa004d
:10b75000000006000800fa00d3ff07000000e00028
:10b760007d003200e0ff0700204798003a08e20021
:10b77000790032002e4090000080fb0030079800d6
:10b78000d0042000be009000808f500026003200c0
:10b79000d0042000be009000808f50000d003c00bf
:10b7a00000032000be009000808f50006a0035002a
:10b7b00090032000be009000808f500033003400c2
:10b7c00050042000be009000808f50002400320002
:10b7d0006100370020052000be009000808f5000df
:10b7e0001100320020052000be009000808f500024
:10b7f00005003c0000052000be009000808f500036
:10b80000090032005400370030052000be009000cf
:10b81000808f50000a00320040052000be009000da
:10b82000808f50004c003a002e4090005eedb70033
:10b83000414d8000108f210010f5070046003700b1
:10b840002001200077fd0700414d8000108f21006e
:10b850000af507000040eb005eedb7003e00370040
:10b86000414d8000a00020000088b90080007800d1
:10b87000108f210001f507003005200069fd070049
:10b880000040eb005eedb700330037002e40900023
:10b890000080fb0001fd2f0001004000e06a8800ed
:10b8a000e06a8000b9fd07005ecdbf000080fb00ac
:10b8b0002007980000052000ae009000808f500007
:10b8c0001200320000052000ae009000808f500072
:10b8d00005003c00d0042000ae009000808f500096
:10b8e0001a0032001c00370020052000ae00900036
:10b8f000808f50001100320040052000ae00900003
:10b90000808f500005003200130037008000eb00ec
:10b91000e06a8000b0fd07000f003700e9e2a800f0
:10b92000cae2a80011002000e06a8000aafd07001a
:10b93000cae2a900e9e2a9000700370011002000cf
:10b94000e06a8000f0fd0700030037008000eb0094
:10b95000e06a8000ecfd07000080fa0000000600ad
:10b960000600fa00881f7800008fbe0070c0b30088
:10b97000504798000040eb00404798004e40900030
:10b98000e74f500016003c005e4090000000fb00b6
:10b9900081d02000010440001e00be00a200200053
:10b9a00003002000dcdd070002c3b300024c4000ae
:10b9b0001e00be00a200200003002000c6dd07001c
:10b9c000008fbe005e4090000040e90050479800a4
:10b9d0004e4090000040e80040479800e7ff3700e5
:10b9e0000040eb0010edb7004f0478000080fa0033
:10b9f000000006000400fa00008fbe001e00be001a
:10ba0000d7ff070008cdbf00c8f0070009cdbf0071
:10ba1000c6f007000acdbf00c4f007000bcdbf0081
:10ba2000c2f007000ccdbf00c0f007000dcdbf0075
:10ba3000bef007000ecdbf00bcf007000fcdbf0069
:10ba4000baf007000080fa00000006000600fa00c5
:10ba500020002000200798006000b800008fbe0082
:10ba6000ae00900020688000808f500019003d00db
:10ba70001e00be00a20020000203b8000001eb007f
:10ba80000282b9000701780004014100a3002000f0
:10ba90000388b90000014100820378002e00900065
:10baa00081cf200001004000104078000000fb0022
:10bab000cf80de006f0060008000eb00001f4300bd
:10bac00001974b002e0090000000e800200798002e
:10bad000e3ff37001e00be000080fa0000000600f1
:10bae0000200fa0060418000008fe9001e00e000c3
:10baf00002003d000000eb00000f78001e007800ff
:10bb0000801f7800e0f12e00801f78002bd2070004
:10bb1000e48757000080fa00000006000000fa00e9
:10bb20003408e20006003a009e08f80050f22e00a9
:10bb3000801f780021d20700e487570005003700f6
:10bb40007608f80050f22e00801f78001bd2070004
:10bb5000e48757000080fa00000006000000fa00a9
:10bb6000104180000000d00001932000010040003f
:10bb700010007800801f7800c0f22e00801f78002f
:10bb80000ed20700e48757000080fa00000006008c
:10bb90000000fa002c09f80030f32e00801f780016
:10bba00006d20700e48757000080fa000000060074
:10bbb0000c00fa00889fbe00f04080000141800028
:10bbc0004f8ade00cfa2de00f040800001418000fd
:10bbd0000401780084017800844c8000954c80003a
:10bbe0004facde00cfc4de00844c8000954c80005a
:10bbf000080378008803780012dd0700200798000a
:10bc00003107980042079800530798002e009000d3
:10bc1000be0090004e019000de0190001402200052
:10bc20008381d1000281d3008180d3000080d300c2
:10bc30000402e900faff3a00008fbe00a0f32e00d4
:10bc4000801f7800ddd107008f87e9001e00be004d
:10bc500068ff0700d0f32e00801f7800d7d10700bf
:10bc60008f87e9004f04be000080fa000000060044
:10bc70000000fa007409f80000f42e00801f78001c
:10bc8000ced10700e48757000080fa0000000600cc
:10bc90000000fa00a04b80000000d000c1972000f7
:10bca00001004000100078006101b900804f2200bf
:10bcb00011002000b3dc0700809fbe0070f42e004e
:10bcc000801f7800bdd10700e68757000080fa008a
:10bcd000000006000000fa006c09f800f0f42e00e5
:10bce000801f7800b5d10700e48757000080fa0074
:10bcf000000006000000fa003408e20005003a00e7
:10bd000060f52e00801f7800acd107008f87e90016
:10bd100004003700c0f52e00801f7800a7d107006f
:10bd20008f87e9000080fa00000006000c00fa008e
:10bd300046ff0700008fbe005000200001002000d9
:10bd40001e0f40005e97480000a02500212620001d
:10bd5000be0f1000ae8f18000300360000a02500b3
:10bd600021262000008fbe001e00be000001eb0057
:10bd70008001eb0024d120005403be004402be0029
:10bd8000b0dc0700200798003107980042079800b0
:10bd90005307980011418000400020000008b800bf
:10bda000c28a2000020240002e009000be009000d7
:10bdb0004e019000de019000f50120008381d1004a
:10bdc0000281d3008180d3000080d3008502e90086
:10bdd000faff3a00008abe000080fa000000060068
:10bde0000200fa00faccbf000000fb006f0f6000f9
:10bdf000200020009e0f10000200340020002000d0
:10be0000000f78001e007800a04b88000080fa0028
:10be1000000006000200fa00881f78000bff0700f0
:10be2000000f7800a04b80000000d000c1972000d8
:10be3000010440001e0078006101b900804f22001b
:10be4000110020004fdc0700000c7800a04b8000a0
:10be50000000d000c197200001014000c1272e0042
:10be6000a04b80000000d0000100400012017800cb
:10be7000900f510009003d00a04b80000000d00051
:10be8000c197200001014000c1272e00a04b800077
:10be90000000d0000100400010097800a04b800095
:10bea0000000d000c19720000101400021282e0091
:10beb000a04b80000000d00001004000120178007b
:10bec000900f510009003400a04b80000000d0000a
:10bed000c19720000101400021282e00a04b8000c6
:10bee0000000d00001004000100978004f047800e5
:10bef0000080fa00000006000200fa00faccbf0041
:10bf00000000fb006f0f6000100020009e0f10006b
:10bf10000200340010002000000f78001e0078009e
:10bf2000604b88000080fa00000006000200fa0062
:10bf300010c3b300fa4ce30002003a00cae2a800c2
:10bf400001003700cae2a9000080fa0000000600e4
:10bf50000200fa000000eb00000f7800b0002000a3
:10bf60009e0f100006003c0080cf20009e00400085
:10bf70000040eb00804878001e0fe800f7ff370014
:10bf80000000eb00206888000080fa000000060036
:10bf90000400fa00004f78001e04e0000c0032009c
:10bfa000a0c0b3009e4f10000900320000c2b300d1
:10bfb0009e4f100006003200c0c2b3009e4f10001a
:10bfc00003003200e0c2b3009e4f100003003a00ad
:10bfd0001000200010079800020037000000eb005e
:10bfe000100798001e0090000080fa000000060074
:10bff0000a00fa006141800030688000808f5000a4
:10c0000007003200f40ce20005003a004006200070
:10c01000a06788006041800030688800b0fe07009b
:10c0200051ef07000000e000c00032005eef0700a3
:10c03000004f78001e407800d5ff07000000e000a8
:10c04000ba003a00d0c3b3009e4f10000300320084
:10c05000f0c3b3009e4f100001003a00bcff070080
:10c06000d1c0b3009ecf1000a6003a00f8ccbf00ac
:10c070000000fb0040079800d0032000ce00900095
:10c08000808f500049003200f0032000ce00900065
:10c09000808f500099003a00f9ccbf000000fb00ef
:10c0a0002007980020052000ae009000808f5000ef
:10c0b0003900320020052000ae009000808f500033
:10c0c00016003c0020042000ae009000808f50003d
:10c0d0002300320020042000ae009000808f50002a
:10c0e00005003c0010042000ae009000808f50003e
:10c0f000250032002b00370060042000ae009000c5
:10c10000808f50001e003200d0042000ae0090004e
:10c11000808f5000160032002200370040052000ba
:10c12000ae009000808f50001d00320040052000be
:10c13000ae009000808f50000b003500600520009d
:10c14000ae009000808f50000b0032007005200080
:10c15000ae009000808f50000d00320011003700bb
:10c160005ffe07000f0037006cfe07000d00370070
:10c170007afe07000b00370085fe07000900370034
:10c180008bfe070007003700b9fe070005003700e7
:10c19000bffe070003003700cefe07000100370096
:10c1a000d4fe07006aff070060003700f9ccbf002b
:10c1b0000000fb003007980020052000be00900022
:10c1c000808f50004800320020052000be00900003
:10c1d000808f500012003c0060042000be009000e0
:10c1e000808f50003a00320060042000be009000b2
:10c1f000808f500005003c0010042000be0090001d
:10c20000808f5000340032003a003700d004200004
:10c21000be009000808f50001300320035003700c0
:10c2200060052000be009000808f50001e0032008c
:10c2300060052000be009000808f500005003c008b
:10c2400040052000be009000808f50002800320082
:10c250002800370070052000be009000808f50003d
:10c260001f00320023003700faccbf000000fb00a3
:10c270006f006000100798001e009000e30f500050
:10c2800002003400300020001007980010418000a8
:10c290000000d00001932000010040009e009000ab
:10c2a0000108780013003700e8fd07001007980028
:10c2b0001e009000f90f5000020034009001200091
:10c2c000100798001e0090006049880009003700a0
:10c2d00096fe070007003700c1fe07000500370083
:10c2e000ccfe07000300370003ff07000100370002
:10c2f0000eff070016ff07000c00370014ff0700b1
:10c300000a0037002068800081cf20000100400033
:10c310001e48780020688000ea0f500003003c00af
:10c32000206880000000e800206888000080fa0093
:04c330000000060003
:020000040000fa
:0200000401f009
:04000000ebfb000016
:020000040000fa
:0200000401f009
:04000400ff7f00007a
:020000040000fa
:0200000401f009
:04000800ffff0000f6
:020000040000fa
:0200000401f009
:04000c00ffff0000f2
:020000040000fa
:0200000401f009
:04001000ffff0000ee
:020000040000fa
:0200000401f009
:04001400ffff0000ea
:020000040000fa
:1000080072440000264300005c43000034440000b2
:100018005a44000072440000724400007244000018
:100028007244000072440000724400004a45000017
:10003800724400007244000072440000b846000098
:10004800c64800001e3e00007244000072440000d2
:1000580072440000724400007244000072440000c0
:1000680072440000724400007244000072440000b0
:1000780072440000724400007244000072440000a0
:10008800a65a000072440000724400007244000046
:100098007244000072440000724400007244000080
:1000a8007244000072440000724400007244000070
:1000b8002c410000a040000072440000724400007f
:1000c8007244000072440000724400007244000050
:1000d8007244000072440000724400007244000040
:1000e8007244000072440000724400007244000030
:0800f800724400007244000094
:020000040000fa
:1001080072440000264300005c43000034440000b1
:100118005a44000072440000724400007244000017
:100128007244000072440000724400004a45000016
:10013800724400007244000072440000b846000097
:10014800c64800001e3e00007244000072440000d1
:1001580072440000724400007244000072440000bf
:1001680072440000724400007244000072440000af
:10017800724400007244000072440000724400009f
:10018800a65a000072440000724400007244000045
:10019800724400007244000072440000724400007f
:1001a800724400007244000072440000724400006f
:1001b8002c410000a040000072440000724400007e
:1001c800724400007244000072440000724400004f
:1001d800724400007244000072440000724400003f
:1001e800724400007244000072440000724400002f
:0801f800724400007244000093
:020000040000fa
:10c3340020760000312e000030360000003100006d
:10c34400392e0000303400002e320000303000005e
:10c35400390000000100000000000000640000003b
:10c3640000000000e80300000000000010270000a7
:10c3740000000000a0860000010000004042000010
:10c384000f0000003000000000000000dd0100008c
:10c3940000000000a4120000000000006aba0000bf
:10c3a4000000000023480000070000005ad10000ec
:10c3b400480000000e740000da0000001be80000d2
:10c3c400b4010000832d0000d8020000065b0000c9
:10c3d400b00500000bb60000600b0000176c0000f5
:10c3e400c1160000abaa0000aa2a00000e740000c7
:10c3f400da0000001be80000b4010000832d0000f7
:10c40400d8020000065b0000b00500000bb6000077
:10c41400600b0000176c0000c1160000222200000f
:10c4240022220000abaa0000aa2a0000b660000085
:10c434000b360000c11600006c4100004a9f00004a
:10c44400f4490000000000000001000000020000a8
:10c4540000030000000400000005000000060000c6
:10c4640000060000000700000007000000070000ad
:10c4740000070000313200003030000020200000ae
:10c4840000000000323400003030000020200000a2
:10c49400000000003438000030300000202000008c
:10c4a4000000000039360000303000002020000079
:10c4b400000000003139000032300000302000005c
:10c4c4000000000033380000343000003020000049
:10c4d4000000000035370000363000003020000036
:10c4e400000000003131000035320000303000001f
:10c4f400200000003a0000002100000012000000ab
:10c50400960000003a000000210000000a0d00001f
:10c51400576f000072640000732000003d2000008b
:10c52400256400002c2000005375000063650000a2
:10c5340073730000203d000020250000642c0000df
:10c544002043000068650000636b00007375000001
:10c554006d2000003d20000025580000000a000066
:10c564000d5700006f72000064730000203d00004e
:10c5740020250000642c0000205300007563000097
:10c584006365000073730000203d00002025000057
:10c59400642c00002043000068650000636b000009
:10c5a400737500006d2000003d2000002558000038
:10c5b4000050000057520000005000005752000085
:10c5c400202d00002e2d00005700000049440000db
:10c5d4000041000000490000442000002d2e00000e
:10c5e4002d2d0000410000005246000020500000a4
:10c5f4006f77000065720000203d000020000000fd
:10c604002064000042000000507700007220000007
:10c614004f4600004620000061660000746500007b
:10c624007220000025690000202000000056000050
:10c63400464f0000206c00006f6300006b20000078
:10c644002020000020200000204f00004e000000a9
:10c65400564600004f2000006c6f0000636b000022
:10c664002020000020200000204f0000464600004b
:10c67400000a00000d5500007365000072200000e0
:10c684007365000074740000696e00006773000035
:10c6940020730000617600006564000020740000cf
:10c6a4006f20000045450000505200004f4d00002f
:10c6b4002c200000506f00007765000072200000fd
:10c6c4006f660000660a00000d000000525300006f
:10c6d40032330000322000005465000073740000ff
:10c6e400202000002020000020200000005700002f
:10c6f40061690000746900006e6700002064000036
:10c7040061740000612e00002e2e00002e00000037
:10c714005258000020640000617400006120000091
:10c72400200000002020000030780000004a0000b3
:10c73400554d0000412d00005452000058320000b5
:10c7440020000000202000004f480000324e00006e
:10c754004c540000204f000048370000535600009e
:10c7640020200000000a00000d0a00000d4a00000d
:10c77400554d0000412d0000545200005832000075
:10c7840020460000697200006d77000061720000ad
:10c7940065200000002c00002042000075690000a4
:10c7a4006c640000200000000a0d0000436f0000cc
:10c7b400707900007269000067680000742000004e
:10c7c4004a75000068610000204e0000696900009d
:10c7d4006e6900006b6f0000736b0000692c000031
:10c7e400204f0000483200004e4c0000540a000064
:10c7f4000d0a00000d00000053790000737400005e
:10c80400656d0000204300006c6f0000636b000046
:10c81400203d000020250000692000006b48000036
:10c824007a0a00000d0000004a5500004d41000046
:10c834002d540000525800003220000055410000e1
:10c844005254000032200000666900007865000040
:10c8540064200000393600003030000020620000ff
:10c86400640a00000d000000506f000077650000ae
:10c87400722000004f4e000000530000657200005b
:10c884007669000063650000204d00006f640000bd
:10c8940065200000202000002000000050750000ea
:10c8a400736800002044000049530000504c00000d
:10c8b40041590000206e0000787400000050000010
:10c8c40075730000682000004641000053540000c6
:10c8d400203d000020530000617600006500000048
:10c8e4000a0d000045450000505200004f4d000065
:10c8f4002063000068650000636b0000737500002e
:10c904006d7300002c200000436100006c200000c7
:10c914003d200000255800002c2000004465000044
:10c924006620000043730000203d00002025000025
:10c93400582c00002046000061630000746f000062
:10c9440072790000206400006566000061750000d3
:10c954006c740000207200006573000065740000b0
:10c96400732000003d20000025640000000a000040
:10c974000d45000045500000524f00004d200000be
:10c9840063680000656300006b730000756d000050
:10c9940020650000727200006f7200002c200000fd
:10c9a400726500006c6f0000616400002066000086
:10c9b40061630000746f000072790000206400005d
:10c9c40065660000617500006c740000730000006f
:10c9d40050750000736800002053000045540000a7
:10c9e400206600006f72000020200000202000005c
:10c9f4000066000061630000746f0000727900003b
:10ca04002064000065660000617500006c7400001d
:10ca1400730000000a0d000053650000742000003c
:10ca2400554100005254000031200000757300008d
:10ca3400657200002062000061750000642000003f
:10ca44007261000074650000207400006f20000013
:10ca540023250000692c000020200000257300001d
:10ca6400626400000a0d0000000a00000d5300007b
:10ca7400657400002055000041520000542000005d
:10ca8400757300006572000020620000617500008b
:10ca940064200000726100007465000020740000ce
:10caa4006f20000023250000692c000020200000d6
:10cab40025730000626400000a0d000000560000a7
:10cac400464f0000412000003d3e0000205600007b
:10cad400464f0000422000006f6b00002000000061
:10cae400564600004f420000203d00003e2000005a
:10caf400564600004f410000206f00006b200000ec
:10cb040000200000564600004f00000020200000d6
:10cb1400004c000053420000005500005342000046
:10cb2400002000004357000000540000756e000010
:10cb34006500000020200000545800000020000080
:10cb44004e41000052000000204d00004944000006
:10cb54000020000057490000440000005357000023
:10cb640052000000204e00002f4100002000000071
:10cb740053570000522000002d2e00002d2d0000e0
:10cb8400002000000056000000230000256c000077
:10cb940058000000205200000020000053700000e4
:10cba4006c740000002000005300000020460000c8
:10cbb400002000005600000020200000204c00004f
:10cbc4006f6300006b00000020410000646a0000f5
:10cbd400757300007400000041470000432000000a
:10cbe4003d20000046610000737400002020000016
:10cbf40020200000202000000041000047430000e6
:10cc0400203d0000205300006c6f000077200000de
:10cc14002020000020200000200000004e410000e1
:10cc2400520000004d490000440000005749000034
:10cc340044000000204c000050460000202000006a
:10cc4400002500006c690000204800007a200000e4
:10cc5400200000004e420000206f000070740000ad
:10cc6400696f00006e2000003d2000004f4e000060
:10cc740020200000004e0000422000006f700000e1
:10cc8400746900006f6e0000203d0000204f00001a
:10cc94004646000020000000537000006565000057
:10cca40063680000507200006f630000203d0000c4
:10ccb400204f00004e20000000530000706500006b
:10ccc4006563000068500000726f0000632000007c
:10ccd4003d2000004f460000460000004146000091
:10cce400206900006e2000003d2000004c69000017
:10ccf4006e6500002020000020200000004100009c
:10cd040046200000696e0000203d0000204d000018
:10cd140069630000202000002020000020000000a3
:10cd24004b65000079650000722000003d20000082
:10cd3400004400006f74000020700000726900005d
:10cd44002e000000496100006d620000696300006c
:10cd54002041000000490000616d0000626900008c
:10cd64006320000042000000537400007261000060
:10cd74006967000068740000004300005720000049
:10cd840070690000746300006820000025690000d9
:10cd9400204800007a2000002000000043570000d3
:10cda400207000006f740000203d0000205300003c
:10cdb40071750000656c00006368000000430000aa
:10cdc40057200000706f0000742000003d20000018
:10cdd40043570000737000006565000064000000a4
:10cde4004c43000044200000424c0000203d000061
:10cdf40020250000692000002020000020200000e1
:10ce040020000000436f00006e7400007261000097
:10ce140073740000203d00002025000069200000fc
:10ce2400200000004c43000044200000546900002e
:10ce34006d650000722000004f460000462000008f
:10ce440020200000004c0000434400002054000057
:10ce5400696d000065720000202500006920000053
:10ce64007320000020200000005200005332000014
:10ce740033320000203d0000200000004a5500002d
:10ce84004d41000054520000583200000059000087
:10ce94006165000073750000434100005400000008
:10cea400566f000069630000654d0000656d000069
:10ceb400005400006573000074200000202000006e
:10cec4002000000042610000756400002052000050
:10ced40061740000653d00002573000000560000e9
:10cee400464f0000203d0000204100002f4200007a
:10cef400202b000020530000706c00007400000020
:10cf0400564600004f2000003d2000002569000027
:10cf1400204d0000656d000020200000202000004e
:10cf240020000000462000002569000020250000a4
:10cf34006920000057200000005200002025000056
:10cf4400692000002569000020570000200000002f
:10cf54002000000000010000010200002003000086
:10cf64000304000004020000060600000606000098
:10cf7400050700000707000086010000c20000004a
:10cf84006100000030000000170000000b000000ea
:10cf940007000000030000000a0d00004f750000a8
:10cfa400745f0000697800006420000025690000b7
:10cfb4002c200000496e00005f69000064780000c6
:10cfc4002025000069200000200a00000d00000058
:10cfd4000a0d000054520000415000003a200000a5
:10cfe4004f730000636900006c610000746f0000ff
:10cff4007220000045720000726f0000720a000087
:10d004000d0000004f530000434300004f4e00004a
:10d014002030000078250000580a00000d000000b0
:10d024000a0d000054520000415000003a20000054
:10d034004164000064720000657300007320000006
:10d0440045720000726f0000720a00000d000000bb
:10d05400573000002030000078250000580a0000f6
:10d064000d0000005731000020300000782500003a
:10d07400580a00000d000000573200002030000064
:10d0840078250000580a00000d0000005733000006
:10d094002030000078250000580a00000d00000030
:10d0a400573400002030000078250000580a0000a2
:10d0b4000d000000573500002030000078250000e6
:10d0c400580a00000d000000573600002030000010
:10d0d40078250000580a00000d00000057370000b2
:10d0e4002030000078250000580a00000d000000e0
:10d0f400573800002030000078250000580a00004e
:10d104000d00000057390000203000007825000091
:10d11400580a00000d0000005731000030200000c4
:10d1240030780000255800000a0d00000057000068
:10d13400313100002030000078250000580a00003a
:10d144000d0000005731000032200000307800004c
:10d15400255800000a0d000000570000313300007c
:10d164002030000078250000580a00000d0000005f
:10d1740057310000342000003078000025580000aa
:10d184000a0d000000570000313500002030000077
:10d1940078250000580a00000d0000000a0d000068
:10d1a40054520000415000003a2000005374000023
:10d1b400616300006b20000045720000726f000084
:10d1c400720a00000d0000000a0d00005452000015
:10d1d400415000003a2000004d61000074680000d6
:10d1e40020450000727200006f7200000a0d0000fa
:10d1f400000a00000d530000707500007269000001
:10d204006f75000073200000496e00007465000013
:10d2140072720000757000007420000045720000f6
:10d22400726f0000720a00000d0000002020000050
:10d234002020000045720000726f00007220000080
:10d244002120000020200000202000000000000019
:10d254000a0d000053650000727600006963000047
:10d264006520000026200000636100006c69000056
:10d274006272000061740000696f00006e2000009b
:10d284006d6f000064650000000a00000d4400009a
:10d2940049530000504c000041590000203d00005b
:10d2a4002070000061720000616d00006574000070
:10d2b4006572000020730000656c00006563000067
:10d2c400742c00002046000041530000542f00003d
:10d2d4005646000041530000542000003d20000049
:10d2e40073610000766500002026000020650000c0
:10d2f4007869000074000000536500007420000089
:10d3040052650000662000004f7300006320000097
:10d314004672000065710000004f00007363000056
:10d32400202500006c690000204800007a000000fd
:10d3340053750000707000006c790000202000001c
:10d34400005600002020000000430000616c000033
:10d35400206d0000756c0000742000003d2000006a
:10d36400256c00006920000020200000200000003f
:10d374004265000065700000206c0000656e0000ce
:10d384002c200000303d00004f46000046200000e5
:10d394000042000065650000702000003d20000090
:10d3a40025690000206d000073200000202000008b
:10d3b40020000000532d00006d650000746500001e
:10d3c40072000000436100006c2000006d750000d5
:10d3d4006c740000203d0000202500006c690000f2
:10d3e40020200000004600006f72000077610000fa
:10d3f400726400002000000052460000204100003a
:10d404006d7000002e2000000050000075730000b5
:10d41400682000004641000053540000206c0000c6
:10d424006f6e0000672000003d0000006661000090
:10d43400637400006f7200007920000064650000ce
:10d4440066610000756c0000747300000046000003
:10d4540061630000746f00007279000020730000a3
:10d464006574000075700000206f00006b00000000
:10d474000a0d000046610000637400006f72000032
:10d48400792000006465000066610000756c00008e
:10d49400747300002072000065730000746f000054
:10d4a4007265000064000000436100006c690000c4
:10d4b400627200002e2000005361000076650000b7
:10d4c400640000000a0d0000436100006c69000064
:10d4d4006272000061740000696f00006e20000039
:10d4e4007365000074740000696e000067730000c7
:10d4f4002073000061760000656400002074000061
:10d504006f20000045450000505200004f4d0000c0
:10d5140000000000447500006d700000204500000c
:10d5240045500000524f00004d200000636f000082
:10d534006e740000656e0000747300000a0d000034
:10d54400000a00000d250000352e000034580000ac
:10d554000020000025340000580000000a0d0000df
:10d564004c610000737400002073000075630000b8
:10d574006365000073730000206300006f640000a3
:10d58400652000003d200000255800002000000018
:10d594000a0d00004a5500004d4100002d540000c2
:10d5a4005258000032200000636f000070790000c0
:10d5b4007269000067680000742000004f48000092
:10d5c4003753000056200000262000004f4800007a
:10d5d400324e00004c5400000a0d0000000a000006
:10d5e4000d5300006f660000747700006172000044
:10d5f400652000007665000072730000696f00000a
:10d604006e200000002c0000206300006f700000fa
:10d61400797200006967000068740000204a000005
:10d6240075680000612000004e690000696e00000a
:10d63400696b00006f7300006b690000204f0000ed
:10d64400483200004e4c0000540a00000d00000057
:10d654000a0d000041440000432000002569000039
:10d66400203d000020250000690000004545000021
:10d67400505200004f4d00002072000065730000fe
:10d6840065740000206300006f7500006e74000074
:10d6940065720000206300006c6500006172000088
:10d6a400656400000a0d0000004c000043440000c3
:10d6b4002077000072690000746500000a0d000004
:10d6c4000063000068610000722000003d2000003b
:10d6d400257800000a0d0000004c000043440000bf
:10d6e4002062000061720000206700007261000087
:10d6f40070680000202600002063000068610000bc
:10d704007261000063740000657200002074000000
:10d7140065730000740a00000d000000256300001a
:10d72400203d000020300000782500005820000033
:10d73400200000000a0d00004d7500007465000013
:10d74400000a00000d41000075640000696f0000cc
:10d75400206f00006e0000000a0d0000535f0000ff
:10d764006d65000074650000722000003d2000001b
:10d77400253100002c5000004f540000203d0000d3
:10d7840020250000690a00000d0000000a0d0000b9
:10d794002065000065700000726f00006d2e0000af
:10d7a4006465000066760000616c00002e7600005f
:10d7b400666f00005f730000656c0000203d000090
:10d7c40020250000690000000a0d000020760000fa
:10d7d400666f00005f69000064780000203d00006f
:10d7e40020250000690000000a0d000020650000eb
:10d7f40065700000726f00006d2e0000646500000b
:10d8040066760000616c00002e6d00006f640000fd
:10d81400655b0000766600006f5f000069640000cd
:10d82400785d0000203d0000202500006900000014
:10d834000a0d00002065000065700000726f000092
:10d844006d2e00006465000066760000616c0000c7
:10d854002e6d00006f640000655b0000325d000007
:10d86400203d000020250000690000000a0d000092
:10d8740020630000775f00006163000074690000aa
:10d8840076650000203d00002025000069000000ae
:10d894000a0d000020740000756e0000655f000032
:10d8a4006f6e0000203d000020250000690000008c
:10d8b4000a0d000020500000545400005f4900008d
:10d8c4004e2000003d20000025690000000a0000f1
:10d8d4000d530000657400003a20000065650000e7
:10d8e400707200006f6d00002e6400006566000019
:10d8f400766100006c2e00006d6f0000646500000e
:10d904005b3200005d2000003d200000000a0000a2
:10d914000d52000065660000204f00007363000094
:10d92400203d0000202500006c690000204d00000f
:10d93400487a00000a0d0000000a00000d6d000086
:10d9440073200000636f0000756e000074650000b2
:10d95400722000003d200000256900000a0d00002f
:10d96400000a00000d53000050490000205400003c
:10d97400780000000a0d0000535000004920000008
:10d9840054780000206300006f6e000074000000f3
:10d994000a0d000050410000204100007474000092
:10d9a400656e000075610000746f00007220000055
:10d9b4003d2000003078000025580000000a0000d7
:10d9c4000d5200004620000041740000746e0000f7
:10d9d40020730000656c0000656300007420000083
:10d9e40069640000782000003d20000025690000e3
:10d9f4002c20000048430000353900003520000089
:10da04006269000074730000203d000020300000b3
:10da140078250000580000000a0d0000444400006e
:10da240053200000747500006e650000207400002f
:10da340065730000742000004f4e0000000a0000cf
:10da44000d4400004453000020740000756e000073
:10da5400652000007465000073740000204f00000e
:10da640066660000000a00000d44000044530000f4
:10da740020740000756e0000696e000067200000cd
:10da8400776f000072640000206400006973000076
:10da9400706c000061790000000a00000d4e000067
:10daa4006f7200006d6100006c200000467200007f
:10dab40065710000756500006e6300007920000048
:10dac40064690000737000006c610000790000005c
:10dad4000a0d000044440000532000007475000047
:10dae4006e6900006e67000020730000746500001a
:10daf400702000002320000025690000203d000064
:10db0400202500006c690000000a00000d4400009c
:10db14006976000020620000792000005a65000048
:10db2400726f0000004b000065790000206900005e
:10db3400733a000020250000640a00000d00000074
:10db440054720000793a000020560000616c000015
:10db540069640000206300006f6d00006d610000c7
:10db64006e640000730a00000d0000001000000045
:10db7400ff03000000040000af040000b004000034
:10db840007050000080500005f05000060050000af
:10db9400b7050000b80500000f06000010060000dd
:10dba4006706000068060000bf060000c00600000b
:10dbb40017070000180700008f0700000a0d000077
:10dbc40054520000582d000032200000766f0000ef
:10dbd40069630000652000006d6500006d6f000042
:10dbe40072790000206f000070740000696f0000fb
:10dbf4006e200000666f0000756e00006420000057
:10dc0400284900005344000031370000323400003a
:10dc1400302000006368000069700000290a0000d9
:10dc24000d000000504c000041590000204d000040
:10dc3400656d0000202300002025000069200000fd
:10dc44002000000054580000204d00002025000052
:10dc54006920000020000000546900006d65000088
:10dc6400202500006920000073200000202000000f
:10dc74002020000020000000524500004320000046
:10dc84004d69000063200000204d0000656d000018
:10dc9400202300002025000069200000005200001d
:10dca400582000004d2000002569000020200000bd
:10dcb400000000000a0d0000566f000069630000b8
:10dcc400652000004d6500006d200000636d0000bc
:10dcd400642000003d200000000a00000d560000f2
:10dce4006f69000063650000204d0000656d000051
:10dcf40020530000746f0000702000006f7000005b
:10dd04006572000061740000696f00006e0000001d
:10dd14000a0d0000566f00006963000065200000d2
:10dd24004d6500006d6f00007279000020650000f1
:10dd34007261000073650000206100006c6c0000db
:10dd4400000a00000d4d0000656d0000203d00003c
:10dd540020250000690000000a0d0000564d000057
:10dd64002c200000706c000061790000206d000020
:10dd7400656d00006f720000790000000a0d00005c
:10dd8400564d00002c20000054580000000a0000ea
:10dd94000d5600004d20000052580000000a0000fb
:10dda4000d5600004d2c0000205200006563000059
:10ddb4006f72000064200000667200006f6d000046
:10ddc400204d000069630000000a00000d560000a9
:10ddd4006f69000063650000204d0000656d000060
:10dde4006f720000792000006f70000074690000f9
:10ddf4006f6e0000206e00006f7400002069000048
:10de04006e730000746100006c6c000065640000b7
:10de1400003f00000000000086010000c200000076
:10de24006100000030000000170000000b0000003b
:10de340007000000030000003d42000025690000c7
:10de44000a0d0000003d000053250000690a00008f
:10de54000d0000003d4d0000256900000a0d000082
:10de6400003d000056250000690a00000d00000076
:10de74003d460000000a00000d0000003d41000086
:10de8400256900000a0d0000003d00005725000030
:10de94006c6900000a0d0000003d000052250000de
:10dea400690a00000d0000003d540000310a000022
:10deb4000d0000003d540000300a00000d00000079
:020000040000fa
:10dec400600d0000020000000200000000000000dd
:10ded40000080000be01000000000000be090000b0
:10dee4000c01000000000000620d000002000000b0
:10def40002000000010000003c0d000006000000cc
:10df040000000000420d00000600000000000000b8
:10df1400be0c00002000000000000000de0c000029
:10df24001a00000000000000480d00000600000078
:10df340000000000120d00001800000000000000a6
:10df4400540d00000400000000000000580d000003
:10df54000400000000000000ca0a000002010000e2
:10df640000000000640d0000020000000200000038
:10df7400010000005c0d000004000000000000002f
:10df8400f80c00001a00000000000000cc0b000098
:10df940088000000020000000100000000f20b00f5
:10dfa400f30bf2000bf20b00f20bf2000be20b008e
:10dfb400000000000000000000000000000000005d
:10dfc4000000000000000000000000000002080043
:10dfd40001011a000c1b0c001a0c1a000c1a0c007c
:10dfe4001a0c0a000c0000000000000000000000f1
:10dff400000000000000000000000000000000001d
:10e004000000020008020200420c43000c420c0013
:10e01400420c42000c420c00320c000000000000d4
:10e0240000000000000000000000000000000000ec
:10e034000000000000000000cc0bf4000b1c0c00de
:10e0440000000000000000000000000000000000cc
:10e054002a0d00001200000002000000202b2d00f9
:10e06400233000000100020000040000080010003a
:10e0740000000000a20d00000800000002000000e3
:10e08400686a6c00747a4c00000000004e0d0000b9
:10e094000600000002000000000000000000020072
:10e0a400660d000002000000000000009c0c00004f
:10e0b4002200000002000000303132003334350009
:10e0c40036373800396162006364650066003000e9
:10e0d4003132330034353600373839004142430099
:10e0e4004445460000000000540c000048000000b5
:10e0f40002000000000000000000000024400000b6
:10e104000000000000005900400000000000000072
:10e1140088c34000000000000084d700974100003d
:10e1240080e0370079c3410043176e0005b5b500a0
:10e13400b8934600f5f93f00e9034f00384d32002b
:10e144001d30f900487782005a3cbf00737fdd0020
:10e154004f157500700d0000320000000200000031
:10e164004e414e00006e61006e0049004e460000b4
:10e17400696e6600003031003233340035363700c2
:10e184003839610062636400656600003031320032
:10e1940033343500363738003941420043444500b2
:10e1a40046000000680d00000200000002000000ac
:10e1b40000000000aa0d00000200000002000000a0
:10e1c400300000006a0d00000200000002000000a0
:10e1d400000000006c0d00000200000002000000be
:10e1e400010000006e0d00000200000000000000ad
:04e1f4000000000027
:00000001FF
